:0200000480007A
:10000000B72F0000938F0F8073900F306F00400365
:100010001300000013000000130000001300000094
:100020001300000013000000130000001300000084
:100030001300000013000000130000001300000074
:100040009702000093824211739052309300000097
:10005000130100009301000013020000930200004E
:100060001303000093030000130400009304000036
:10007000130500009305000013060000930600001E
:100080001307000093070000130800009308000006
:100090001309000093090000130A0000930A0000EE
:1000A000130B0000930B0000130C0000930C0000D6
:1000B000130D0000930D0000130E0000930E0000BE
:1000C000130F0000930F000097110200938101B2FB
:1000D00017050200130505339795030093854565C1
:1000E00013060000EF00001A170502001305452F44
:1000F000970502009385452F13060000EF00801836
:1001000017A503001305056397B5030093854562A2
:1001100037B6ABAB1306B6BAEF00C01617B1030083
:1001200013014161EF70005E9392120093D21200AE
:100130009382D2FF638A02008322010013014100EF
:100140006F0000177300203083220100130141006B
:10015000730020301301C1FF23205100F32220340B
:10016000E3C402FC8322010013014100130141F8A2
:1001700023221100232421002326310023284100BB
:10018000232A5100232C6100232E71002320810299
:10019000232291022324A1022326B1022328C10293
:1001A000232AD102232CE102232EF1022320010570
:1001B0002322110523242105232631052328410567
:1001C000232A5105232C6105232E71052320810745
:1001D000232291072324A1072326B1072328C1073F
:1001E000232AD107232CE107232EF107732520347E
:1001F000F3251034130601006F000000731015344E
:1002000083204100032181008321C10003220101D9
:1002100083224101032381018323C10103240102BD
:1002200083244102032581028325C10203260103A1
:1002300083264103032781038327C1030328010485
:1002400083284104032981048329C104032A010569
:10025000832A4105032B8105832BC105032C01064D
:10026000832C4106032D8106832DC106032E010731
:10027000832E4107032F8107832FC1071301C10775
:10028000730020302320C5006376B50013054500B8
:100290006FF05FFF678000000000000000000000BA
:1002A000000000000000000000000000000000004E
:1002B000130101F8232011002322210023243100FF
:1002C0002326410023285100232A6100232C71009A
:1002D000232E8100232091022322A1022324B10294
:1002E0002326C1022328D102232AE102232CF10272
:1002F000232E010323201105232221052324310568
:100300002326410523285105232A6105232C710545
:10031000232E8105232091072322A1072324B1073F
:100320002326C1072328D107232AE107232CF1071D
:100330009702020083A2C20A23A02200F3221034F3
:10034000232E5106EF0080461701020003214109C8
:10035000032101008322C10773901234B7220000E9
:100360009382028873A00230832001000322C1001F
:100370008322010103234101832381010324C1015D
:100380008324010203254102832581020326C10241
:100390008326010303274103832781030328C10325
:1003A000832801040329410483298104032AC10409
:1003B000832A0105032B4105832B8105032CC105ED
:1003C000832C0106032D4106832D8106032EC106D1
:1003D000832E0107032F4107832F81071301010893
:1003E00073002030970202009382C20123A0120002
:1003F00023A2220023A4320023A6420023A85200F5
:1004000023AA620023AC720023AE820023A09202D2
:1004100023A2A20223A4B20223A6C20223A8D202CC
:1004200023AAE20223ACF20223AE020323A01205A8
:1004300023A2220523A4320523A6420523A85205A0
:1004400023AA620523AC720523AE820523A092077E
:1004500023A2A20723A4B20723A6C20723A8D20778
:1004600023AAE20723ACF207EF70C00F17010200C6
:10047000032101F7032101008322C1077390123485
:10048000B72200009382028873A00230832001000B
:100490000322C1008322010103234101832381013F
:1004A0000324C10183240102032541028325810223
:1004B0000326C10283260103032741038327810307
:1004C0000328C103832801040329410483298104EB
:1004D000032AC104832A0105032B4105832B8105CF
:1004E000032CC105832C0106032D4106832D8106B3
:1004F000032EC106832E0107032F4107832F810797
:10050000130101087300203097020200938282EFEA
:1005100083A0020003A1420083A1820003A2C200C3
:1005200083A2020103A3420183A3820103A4C201A7
:1005300083A4020203A5420283A5820203A6C2028B
:1005400083A6020303A7420383A7820303A8C2036F
:1005500083A8020403A9420483A9820403AAC20453
:1005600083AA020503AB420583AB820503ACC20537
:1005700083AC020603AD420683AD820603AEC2061B
:1005800083AE020703AFC20983AF82076780000012
:1005900073700430130101F823201100232221007D
:1005A000232431002326410023285100232A6100FF
:1005B000232C7100232E8100232091022322A102EB
:1005C0002324B1022326C1022328D102232AE102D7
:1005D000232CF102232E01032320110523222105C0
:1005E000232431052326410523285105232A6105AB
:1005F000232C7105232E8105232091072322A10797
:100600002324B1072326C1072328D107232AE10782
:10061000232CF1079702020083A282DC23A0220090
:10062000232E1106EF20D05817010200032141DBD1
:10063000032101008322C10773901234B722000006
:100640009382028873A00230832001000322C1003C
:100650008322010103234101832381010324C1017A
:100660008324010203254102832581020326C1025E
:100670008326010303274103832781030328C10342
:10068000832801040329410483298104032AC10426
:10069000832A0105032B4105832B8105032CC1050A
:1006A000832C0106032D4106832D8106032EC106EE
:1006B000832E0107032F4107832F810713010108B0
:1006C0007300203097070200938747D203A70700E3
:1006D0009307F0FF6306F700737004306F000000AB
:1006E000737004306F000000130101FF2326A10086
:1006F0008327C100739047301300000013010101EC
:1007000067800000130101FFF32740302326F1002A
:1007100073F043308327C1001385070013010101E3
:1007200067800000130101FF2326A1002324B100EC
:100730002322C1008327C1009387C7FF2326F1002E
:10074000032781008327C10023A0E7008327C1007E
:10075000938787FA2326F100032741008327C100EE
:1007600023A0E7008327C100938787FE2326F1009B
:1007700093870100138707008327C10023A0E700A8
:100780008327C100938747FF2326F1001707000046
:10079000130787F38327C10023A0E7008327C10045
:1007A000138507001301010167800000130101FF99
:1007B00023261100EF609050EF20101693070500DC
:1007C00063840700EF20D03E130000008320C100A7
:1007D0001301010167800000130101FF2326A1001E
:1007E0008327C100138787008327C10023A2E70066
:1007F0008327C1001307F0FF23A4E7008327C1006C
:10080000138787008327C10023A6E7008327C10041
:10081000138787008327C10023A8E7008327C1002F
:1008200023A00700130000001301010167800000EE
:10083000130101FF2326A1008327C10023A807007D
:10084000130000001301010167800000130101FE85
:100850002326A1002324B1008327C10083A74700DA
:10086000232EF100832781000327C10123A2E70083
:100870008327C10103A787008327810023A4E70002
:100880008327C10183A787000327810023A2E700F4
:100890008327C1010327810023A4E7008327810068
:1008A0000327C10023A8E7008327C10083A707000F
:1008B000138717008327C10023A0E700130000005F
:1008C0001301010267800000130101FE2326A1002D
:1008D0002324B1008327810083A70700232CF10084
:1008E000032781019307F0FF631AF7008327C100F4
:1008F00083A70701232EF1006F0040038327C10067
:1009000093878700232EF1006F0000018327C10128
:1009100083A74700232EF1008327C10183A7470047
:1009200083A7070003278101E372F7FE8327C10134
:1009300003A747008327810023A2E70083278100C4
:1009400083A747000327810023A4E70083278100B2
:100950000327C10123A4E7008327C10103278100E6
:1009600023A2E700832781000327C10023A8E70013
:100970008327C10083A70700138717008327C100BF
:1009800023A0E700130000001301010267800000AC
:10099000130101FE2326A1008327C10083A70701BD
:1009A000232EF1008327C10083A747000327C1003E
:1009B0000327870023A4E7008327C10083A78700BC
:1009C0000327C1000327470023A2E7008327C101B3
:1009D00083A747000327C100631AF7008327C100DC
:1009E00003A787008327C10123A2E7008327C10053
:1009F00023A807008327C10183A707001387F7FFF8
:100A00008327C10123A0E7008327C10183A7070033
:100A1000138507001301010267800000130101FD27
:100A200023261102232481022326A1002324B100BE
:100A30008327C100232EF1008327C101639607009D
:100A4000737004306F000000EF3010418327C10144
:100A500003A407008327C10103A7C7038327C1019C
:100A600083A707049385070013050700EF80502F25
:100A7000930705003307F4008327C10123A2E70091
:100A80008327C10123AC07028327C10103A7070005
:100A90008327C10123A4E7008327C10103A4070022
:100AA0008327C10183A7C7031387F7FF8327C101EA
:100AB00083A707049385070013050700EF80502ADA
:100AC000930705003307F4008327C10123A6E7003D
:100AD0008327C1011307F0FF23A2E7048327C10185
:100AE0001307F0FF23A4E70483278100639A07021A
:100AF0008327C10183A70701638407048327C101FA
:100B00009387070113850700EF20504C130705005A
:100B1000930710006316F702EFF09FA76F004002E3
:100B20008327C1019387070113850700EFF0DFCA10
:100B30008327C1019387470213850700EFF0DFC9C0
:100B4000EF30903593071000138507008320C10212
:100B5000032481021301010367800000130101FDDA
:100B6000232611022326A1002324B10093070600A7
:100B7000A303F100232C01008327C1006396070023
:100B8000737004306F0000008327810063960700B4
:100B9000232E01006F00C001832581000325C100C1
:100BA000EF80101C9307050093871700232EF10098
:100BB0008327C1019387470513850700EF50D00AAB
:100BC000232AA1008327410163820706832781002E
:100BD000639A0700832741010327410123A0E7000F
:100BE0006F00400183274101138747058327410197
:100BF00023A0E700832741010327C10023AEE702BA
:100C0000832741010327810023A0E70493051000F7
:100C100003254101EFF09FE0832741010347710065
:100C20002388E70483274101232CF10083278101D6
:100C300063960700737004306F0000008327810102
:100C4000138507008320C1021301010367800000A0
:100C5000130101FD2326110293070500A307F100EC
:100C600013054005EF505000232EA1008327C1013A
:100C7000638C07088327C10123A207008327C101D2
:100C800023A007008327C10123A407008327C101F4
:100C900023A607008327C10123AC07028327C101D4
:100CA0001307100023AEE7028327C10123A0070426
:100CB0008327C1011307F0FF23A2E7048327C101A3
:100CC0001307F0FF23A4E7048327C1010347F100C2
:100CD0002388E7048327C101938707011385070051
:100CE000EFF09FAF8327C101938747021385070069
:100CF000EFF09FAE9306000013060000930500007E
:100D00000325C101EF00001E8327C10113850700E1
:100D10008320C1021301010367800000130101FD5C
:100D200023261102232481022326A1008327C10048
:100D3000232CF10083278101639607007370043030
:100D40006F0000008327810103A44700EF3000609B
:100D5000930705006312F4048327810183A7C7006A
:100D60001387F7FF8327810123A6E70083278101EB
:100D700083A7C700639C07009306000013060000CA
:100D80009305000003258101EF00C01593071000B3
:100D9000232EF1006F008000232E01008327C10164
:100DA000138507008320C10203248102130101037C
:100DB00067800000130101FD232611022324810214
:100DC0002326A1002324B1008327C100232CF10096
:100DD0008327810163960700737004306F00000061
:100DE0008327810103A44700EF3040569307050095
:100DF0006312F4028327810183A7C70013871700BA
:100E00008327810123A6E70093071000232EF1001A
:100E10006F00C003930600000326810093050000C5
:100E200003258101EF00C058232EA1000327C10133
:100E300093071000631CF7008327810183A7C70075
:100E4000138717008327810123A6E7008327C101A9
:100E5000138507008320C1020324810213010103CB
:100E600067800000130101FD232611022326A10043
:100E70002324B1008327C1006396070073700430F8
:100E80006F000000032781008327C10063F6E7009D
:100E9000737004306F0000001306200093050000FB
:100EA0000325C100EFF09FCB232EA1008327C101B2
:100EB000638807008327C1010327810023ACE70271
:100EC0008327C10163960700737004306F00000030
:100ED0008327C101138507008320C1021301010389
:100EE00067800000130101FC232E11022326A100BC
:100EF0002324B1002322C1002320D1002326010294
:100F00008327C1002324F10283278102639607000F
:100F1000737004306F00000083278100639807001E
:100F20008327810283A707046396070093071000B5
:100F30006F00800093070000639607007370043011
:100F40006F0000000327010093072000631AF700D9
:100F50008327810203A7C703930710006316F700D6
:100F6000930710006F00800093070000639607004E
:100F7000737004306F000000EF30803F930705006E
:100F800063960700832741006396070093071000CC
:100F90006F008000930700006396070073700430B1
:100FA0006F000000EF30406B8327810203A78703A7
:100FB0008327810283A7C7036368F7000327010023
:100FC000930720006310F7060326010083258100A4
:100FD00003258102EF00101C2322A1028327810236
:100FE00083A747026384070283278102938747020E
:100FF00013850700EF20807D13070500930710007D
:10100000631CF700EFF0CFD86F0000018327410287
:1010100063840700EFF0CFD7EF300068930710002C
:101020006F00400F8327410063980700EF30C066D0
:10103000930700006F00000E8327C102639C070026
:101040009307C10113850700EF20501D930710007F
:101050002326F102EF304064EF10D049EF30C05F3B
:101060008327810203A747049307F0FF6316F70065
:101070008327810223A207048327810203A7870411
:101080009307F0FF6316F7008327810223A4070468
:10109000EF308060130741009307C10193050700FB
:1010A00013850700EF20501C93070500639C07047D
:1010B00003258102EF00504693070500638C070269
:1010C00083278102938707010327410093050700C7
:1010D00013850700EF20004A03258102EF00902CC2
:1010E000EF10904393070500E39E07EAEFF04FCA25
:1010F0006FF05FEB03258102EF00D02AEF10D041A3
:101100006FF05FEA03258102EF00D029EF10D04095
:1011100093070000138507008320C1031301010416
:1011200067800000130101FD232611022326A10080
:101130002324B1002322C1002320D1008327C10032
:10114000232CF1008327810163960700737004301C
:101150006F000000832781006398070083278101C7
:1011600083A7070463960700930710006F008000B1
:101170009307000063960700737004306F0000004F
:101180000327010093072000631AF70083278101DA
:1011900003A7C703930710006316F7009307100017
:1011A0006F0080009307000063960700737004309F
:1011B0006F000000EFF00FD593070500232AF10020
:1011C0008327810103A787038327810183A7C7039F
:1011D0006368F70003270100930720006310F708F6
:1011E000032601008325810003258101EF00807A19
:1011F0008327810103A787049307F0FF6310F70497
:101200008327810183A74702638407048327810121
:101210009387470213850700EF20405B9307050083
:101220006388070283274100638407028327410004
:101230001307100023A0E7006F00800183278101BE
:1012400083A78704138717008327810123A4E7045A
:1012500093071000232EF1006F008000232E010061
:101260008327410113850700EFF00FC88327C101D1
:10127000138507008320C10213010103678000006A
:10128000130101FD232611022326A1002324B1000E
:101290008327C100232CF100832781016396070077
:1012A000737004306F0000008327810183A7070457
:1012B00063860700737004306F000000832781018C
:1012C00083A70700639807008327810183A747004E
:1012D00063960700930710006F00800093070000DB
:1012E00063960700737004306F000000EFF08FC149
:1012F00093070500232AF1008327810103A78703B1
:101300008327810183A7C7036372F70883278101BD
:1013100083A78703138717008327810123ACE70284
:101320008327810103A787049307F0FF6310F70465
:101330008327810183A747026384070483278101F0
:101340009387470213850700EF2040489307050065
:101350006388070283278100638407028327810053
:101360001307100023A0E7006F008001832781018D
:1013700083A78704138717008327810123A4E70429
:1013800093071000232EF1006F008000232E010030
:101390008327410113850700EFF00FB58327C101B3
:1013A000138507008320C102130101036780000039
:1013B000130101FC232E11022326A1002324B100D6
:1013C0002322C1002320D100232601028327C1004C
:1013D0002324F1028327810263960700737004308F
:1013E0006F00000083278100639807008327810234
:1013F00083A7070463960700930710006F0080001F
:101400009307000063960700737004306F000000BC
:10141000EF201076930705006396070083274100AD
:1014200063960700930710006F0080009307000089
:1014300063960700737004306F000000EF30C02126
:101440008327810283A787036382070C8327810296
:1014500083A7C7002322F10283258100032581028F
:10146000EF00806B832701006392070683278102C8
:1014700083A787031387F7FF8327810223ACE70243
:101480008327810283A70700639A0700EF30802B30
:10149000130705008327810223A2E7008327810227
:1014A00083A70701638E07048327810293870701BF
:1014B00013850700EF208031130705009307100004
:1014C0006310F704EFF0CF8C6F0080038327810255
:1014D0000327410223A6E7008327810283A747024F
:1014E00063800702832781029387470213850700E1
:1014F000EF20C02D9307050063840700EFF04F89AC
:10150000EF308019930710006F008011832741008E
:1015100063980700EF304018930700006F004010F9
:101520008327C102639C07009307C101138507004D
:10153000EF20C04E930710002326F102EF30C015B4
:10154000EF10407BEF3040118327810203A747044F
:101550009307F0FF6316F7008327810223A2070495
:101560008327810203A787049307F0FF6316F70020
:101570008327810223A40704EF30001213074100E0
:101580009307C1019305070013850700EF20C04DA5
:1015900093070500639E070603258102EF00406F55
:1015A00093070500638E07048327810283A7070042
:1015B000639E0700EF30400A8327810283A747001C
:1015C00013850700EF20D05FEF30000D83278102E5
:1015D00093874702032741009305070013850700FF
:1015E000EF10507903258102EF00C05BEF10C0724D
:1015F00093070500E39407E4EFE09FF96FF01FE421
:1016000003258102EF00005AEF1000716FF01FE315
:1016100003258102EF000059EF10007093070000CE
:10162000138507008320C1031301010467800000B4
:10163000130101FD232611022326A1002324B1005A
:101640002322C1008327C100232CF10083278101BD
:1016500063960700737004306F00000083278100D9
:10166000639807008327810183A707046396070017
:10167000930710006F008000930700006396070037
:10168000737004306F000000EFF0CF879307050000
:10169000232AF1008327810183A787036388070832
:1016A0008325810003258101EF0000478327810105
:1016B00083A787031387F7FF8327810123ACE70202
:1016C0008327810103A747049307F0FF6310F70402
:1016D0008327810183A7070163840704832781018E
:1016E0009387070113850700EF20400E930705003D
:1016F0006388070283274100638407028327410030
:101700001307100023A0E7006F00800183278101E9
:1017100083A74704138717008327810123A2E704C7
:1017200093071000232EF1006F008000232E01008C
:101730008327410113850700EFE01FFB8327C101C9
:10174000138507008320C102130101036780000095
:10175000130101FD232611022326A1002324B10039
:101760008327C100232CF1008327810163960700A2
:10177000737004306F0000008327810063980700B6
:101780008327810183A7070463960700930710004E
:101790006F008000930700006396070073700430A9
:1017A0006F0000008327810183A707046396070069
:1017B000737004306F000000EFE0DFF49307050062
:1017C000232AF1008327810183A78703638A070205
:1017D0008327810183A7C7002328F1008325810087
:1017E00003258101EF004033832781010327010195
:1017F00023A6E70093071000232EF1006F0080005E
:10180000232E01008327410113850700EFE0DFED60
:101810008327C101138507008320C102130101033F
:1018200067800000130101FD232611022326A10079
:101830008327C10063960700737004306F000000B7
:10184000EF2090618327C10083A78703232EF10037
:10185000EF2090648327C101138507008320C10214
:101860001301010367800000130101FD232611020B
:101870002326A1008327C100232EF1008327C10165
:1018800063960700737004306F000000EF20D05C97
:101890008327C10103A7C7038327C10183A7870348
:1018A000B307F740232CF100EF20105F832781015D
:1018B000138507008320C102130101036780000024
:1018C000130101FE2326A1008327C10063960700B0
:1018D000737004306F0000008327C10083A7870363
:1018E000232EF1008327C101138507001301010294
:1018F00067800000130101FD232611022326A100A9
:101900008327C100232EF1008327C10163960700BE
:10191000737004306F0000000325C101EF004052D6
:101920000325C101EF401054130000008320C102C1
:101930001301010367800000130101FF2326A100AA
:101940008327C10083A7C704138507001301010182
:1019500067800000130101FF2326A1002324B100AA
:101960008327C1000327810023A6E704130000009A
:101970001301010167800000130101FF2326A1006C
:101980008327C10083C707051385070013010101E1
:1019900067800000130101FD232611022326A10008
:1019A0002324B1002322C100232E01008327C1007C
:1019B00083A70704639807028327C10083A7070052
:1019C000639807128327C10083A747001385070088
:1019D000EF20D034232EA1008327C10023A20700CB
:1019E0006F00001183274100639407068327C1001D
:1019F00003A787008327C10083A707041386070076
:101A00008325810013050700EF40905C8327C10008
:101A100003A787008327C10083A707043307F700C4
:101A20008327C10023A4E7008327C10003A7870001
:101A30008327C10083A74700636CF70A8327C1008F
:101A400003A707008327C10023A4E7006F00400A13
:101A50008327C10003A7C7008327C10083A707040A
:101A6000138607008325810013050700EF405056B9
:101A70008327C10003A7C7008327C10083A70704EA
:101A8000B307F0403307F7008327C10023A6E70020
:101A90008327C10003A7C7008327C10083A70700CE
:101AA0006372F7028327C10003A747008327C100A1
:101AB00083A70704B307F0403307F7008327C1006B
:101AC00023A6E70003274100930720006312F702D3
:101AD0008327C10083A78703638C07008327C10086
:101AE00083A787031387F7FF8327C10023ACE7028F
:101AF0008327C10083A78703138717008327C100AB
:101B000023ACE7028327C101138507008320C102AC
:101B10001301010367800000130101FE232E110051
:101B20002326A1002324B1008327C10083A7070433
:101B3000638207068327C10003A7C7008327C1006C
:101B400083A707043307F7008327C10023A6E70014
:101B50008327C10003A7C7008327C10083A74700CD
:101B6000636AF7008327C10003A707008327C1002A
:101B700023A6E7008327C10003A7C7008327C1006E
:101B800083A7070413860700930507000325810038
:101B9000EF401044130000008320C1011301010233
:101BA00067800000130101FE232E11002326A100EF
:101BB000EF20902A6F0000048327C10083A747020B
:101BC000638207048327C1009387470213850700B8
:101BD000EF10D03F9307050063840700EF10D07823
:101BE0008327C10083A787041387F7FF8327C100DA
:101BF00023A4E7048327C10083A78704E34EF0FAF8
:101C00006F008000130000008327C1001307F0FF5E
:101C100023A4E704EF205028EF2010246F000004D5
:101C20008327C10083A70701638207048327C100BC
:101C30009387070113850700EF10503993070500BC
:101C400063840700EF1050728327C10083A7470405
:101C50001387F7FF8327C10023A2E7048327C1006E
:101C600083A74704E34EF0FA6F00800013000000E2
:101C70008327C1001307F0FF23A2E704EF20D02140
:101C8000130000008320C1011301010267800000DE
:101C9000130101FD232611022326A100EF20D01BF2
:101CA0008327C10083A78703639807009307100069
:101CB000232EF1006F008000232E0100EF20D01DA5
:101CC0008327C101138507008320C102130101038B
:101CD00067800000130101FE2326A1008327C100B5
:101CE00063960700737004306F0000008327C10003
:101CF00083A787036398070093071000232EF10042
:101D00006F008000232E01008327C1011385070087
:101D10001301010267800000130101FD2326110257
:101D20002326A100EF2050138327C10003A78703B8
:101D30008327C10083A7C7036318F7009307100028
:101D4000232EF1006F008000232E0100EF20D0141D
:101D50008327C101138507008320C10213010103FA
:101D600067800000130101FE2326A1008327C10024
:101D700063960700737004306F0000008327C10072
:101D800003A787038327C10083A7C7036318F7004E
:101D900093071000232EF1006F008000232E010016
:101DA0008327C1011385070013010102678000002A
:101DB000130101FE2326A1002324B100232E0100DC
:101DC0006F008006178703001307C7928327C1019E
:101DD00093973700B307F70083A7070063900704C2
:101DE00017870300130707918327C10193973700D3
:101DF000B307F7000327810023A0E700178703003C
:101E00001307478F8327C10193973700B307F70064
:101E10000327C10023A2E7006F00C0018327C1018F
:101E200093871700232EF1000327C1019307700049
:101E3000E3FAE7F8130000001301010267800000D5
:101E4000130101FE2326A100232E01006F00C00410
:101E5000178703001307078A8327C1019397370069
:101E6000B307F70083A747000327C1006310F702F9
:101E700017870300130707888327C101939737004B
:101E8000B307F70023A007006F00C0018327C1013B
:101E900093871700232EF1000327C10193077000D9
:101EA000E3F8E7FA13000000130101026780000065
:101EB000130101FD232611022326A1002324B100D2
:101EC0002322C1008327C100232EF100EF20C07818
:101ED0008327C10103A747049307F0FF6316F700A8
:101EE0008327C10123A207048327C10103A7870415
:101EF0009307F0FF6316F7008327C10123A40704AB
:101F0000EF2080798327C10183A78703639E0700A1
:101F10008327C1019387470203264100832581005F
:101F200013850700EF10007F0325C101EFF09FC765
:101F3000130000008320C102130101036780000029
:101F4000130101FC232E1102232EA100232CB1002A
:101F50002328D1002326E1002324F10023220101BC
:101F60002320110193070600231BF1008327C101E1
:101F700063960700737004306F0000000327C100F0
:101F80009307900063F6E700737004306F00000061
:101F9000835761018325410013850700EF10D07E30
:101FA0002324A102832781026386071C83278102E1
:101FB00003A7070383566101B70700409387F7FF24
:101FC000B387F60093972700B307F7002322F102A7
:101FD0008327410293F7C7FF2322F102832741029F
:101FE00093F7370063860700737004306F000000BA
:101FF0008357610113870700832601000326C10070
:102000008325810103258102EF1050410326010140
:102010008325C10103254102EFE0CFF0130705003E
:102020008327810223A0E7008327810063880700BC
:10203000832781000327810223A0E700EF20C061EE
:1020400097E701009387475783A707001387170077
:1020500097E701009387475623A0E70097E7010021
:102060009387073883A707006398070297E7010063
:10207000938707370327810223A0E70097E7010032
:102080009387875303A70700930710006312F70491
:10209000EF10904B6F00C00397E7010093878752C2
:1020A00083A707006396070297E7010093874733EA
:1020B00083A7070083A7C7020327C100636AF7004D
:1020C00097E701009387C7310327810223A0E70028
:1020D00097E701009387075083A70700138717002E
:1020E00097E701009387074F23A0E70097E70100D8
:1020F0009387474E03A707008327810223A4E704A1
:102100008327810203A7C70297E701009387474B04
:1021100083A7070063FCE7008327810203A7C702A8
:1021200097E701009387C74923A0E700832781022F
:1021300003A7C7029307070093972700B387E70019
:102140009397270017E70100130787333387E700CA
:1021500083278102938747009385070013050700B3
:10216000EFE0CFEE930710002326F102EF20C052DC
:102170006F00C0009307F0FF2326F1020327C1027E
:10218000930710006318F70297E7010093878743CE
:1021900083A707006380070297E70100938747241E
:1021A00083A7070083A7C7020327C10063F4E700E2
:1021B000EFE00FBE8327C102138507008320C10310
:1021C0001301010467800000130101FD23261102A1
:1021D0002326A100EF2040488327C100639A07000F
:1021E00097E701009387C71F83A707006F00800050
:1021F0008327C100232EF1008327C1019387470065
:1022000013850700EFE0CFF88327C10183A787027A
:10221000638A07008327C10193878701138507001D
:10222000EFE00FF78327C1019387470093850700ED
:1022300017E5010013058535EFE04FE197E7010051
:102240009387073683A707001387170097E70100D6
:102250009387073523A0E70097E701009387873727
:1022600083A707001387170097E701009387873636
:1022700023A0E700EF20404297E7010093878734CF
:1022800083A707006382070497E701009387471538
:1022900083A707000327C1016312F70297E7010034
:1022A0009387C73383A707006386070073700430E2
:1022B0006F000000EFE0CFAD6F000001EF20C039EC
:1022C000EF208001EF20403D130000008320C10279
:1022D0001301010367800000130101FD2326110291
:1022E0002326A1002324B100232E01008327C1004F
:1022F00063960700737004306F000000832781002D
:1023000063960700737004306F00000097E70100C8
:102310009387C72C83A70700638607007370043078
:102320006F000000EF00101D97E701009387072959
:1023300083A70700232CF1008327C10083A7070090
:1023400003278100B307F700232AF1008327C10088
:1023500083A70700032781016376F7028327C10063
:1023600083A70700032741016370F7040327410196
:102370008327810163FAE70293071000232EF100FF
:102380006F0080028327C10083A707000327410154
:102390006368F700032741018327810163F6E700A3
:1023A00093071000232EF1008327C100032741016A
:1023B00023A0E7008327C1016382070297E701009A
:1023C0009387070283A707009387470013850700B9
:1023D000EFE00FDC03254101EF10502FEF00D01389
:1023E0002328A1008327010163940700EFE04F9A9F
:1023F000130000008320C102130101036780000065
:10240000130101FD232611022326A100232E010022
:102410008327C1006380070697E701009387071CA5
:1024200083A7070063860700737004306F00000005
:10243000EF00500C97E701009387471883A7070028
:102440000327C100B307F700232CF10097E7010031
:10245000938707F983A70700938747001385070031
:10246000EFE00FD303258101EF105026EF00D00AD3
:10247000232EA1008327C10163940700EFE04F9151
:10248000130000008320C1021301010367800000D4
:10249000130101FD232611022326A1008327C10079
:1024A000232CF100832781016396070073700430A9
:1024B0006F00000097E70100938787F283A707006A
:1024C000032781016316F700232E01006F00400AE5
:1024D000EF2080188327810183A74701232AF10079
:1024E000EF20801B97E701009387870883A70700E9
:1024F00003274101630CF70097E7010093878707E3
:1025000083A70700032741016318F7009307200002
:10251000232EF1006F00C0050327410197E701005A
:10252000938747086314F7028327810183A78702F3
:102530006398070093073000232EF1006F004003DB
:1025400093072000232EF1006F0080020327410132
:1025500097E70100938787036318F700930740000C
:10256000232EF1006F00C00093071000232EF1000E
:102570008327C101138507008320C10213010103D2
:1025800067800000130101FD232611022326A1000C
:10259000EF20800C8327C100639A070097E70100B2
:1025A000938707E483A707006F0080008327C1009B
:1025B000232EF1008327C10183A7C702232CF1003A
:1025C000EF20800D83278101138507008320C1023E
:1025D0001301010367800000130101FD232611028E
:1025E0002326A100EFE00F9293070500232EF100B0
:1025F0008327C100639A070097E70100938747DEAE
:1026000083A707006F0080008327C100232CF100FF
:102610008327810183A7C702232AF1008327C101F1
:1026200013850700EFE04F8C8327410113850700D6
:102630008320C1021301010367800000130101FD23
:10264000232611022326A1002324B100232E0100FA
:10265000032781009307900063F6E700737004304E
:102660006F000000032781009307900063F6E700E6
:10267000930790002324F100EF10107E8327C10000
:10268000639A070097E70100938787D583A7070020
:102690006F0080008327C100232CF1008327810174
:1026A00083A70705232AF10003274101832781001F
:1026B000630EF716032781008327410163FEE702BB
:1026C00097E701009387C7D183A7070003278101FC
:1026D0006302F70497E70100938787D083A7070079
:1026E00083A7C702032781006366F70293071000E0
:1026F000232EF1006F00000297E70100938747CE79
:1027000083A70700032781016316F70093071000D2
:10271000232EF1008327810183A7C7022328F1001C
:102720008327810103A707058327810183A7C702A8
:102730006318F700832781010327810023A6E7029E
:10274000832781010327810023A8E70483278101D0
:1027500083A7870163CC07001307A00083278100AC
:102760003307F7408327810123ACE70083278101EA
:1027700083A64701032701019307070093972700CA
:10278000B387E7009397270017E70100130747CFA8
:10279000B387E7006396F600930710006F00800090
:1027A00093070000638C0706832781019387470006
:1027B00013850700EFE0CF9D8327810103A7C702A0
:1027C00097E701009387C7DF83A7070063FCE70053
:1027D0008327810103A7C70297E70100938747DE9C
:1027E00023A0E7008327810103A7C70293070700FF
:1027F00093972700B387E7009397270017E7010017
:10280000130707C83387E7008327810193874700B1
:102810009385070013050700EFE04F830327C101ED
:10282000930710006314F700EFD09FD6EF10D06627
:10283000130000008320C102130101036780000020
:10284000130101FD232611022326A100EF10D06001
:102850008327C100639A070097E70100938747B871
:1028600083A707006F0080008327C100232EF1009B
:102870008327C1019387470013850700EFE04F913D
:102880008327C10183A78702638A07008327C101C9
:102890009387870113850700EFE08F8F8327C1019E
:1028A000938747009385070017E50100130585CF3F
:1028B000EFD0DFF9EF10505E97E70100938747B242
:1028C00083A707000327C1016314F70697E70100F8
:1028D000938747CF83A707006382070297E701002A
:1028E0009387C7CF83A70700638607007370043000
:1028F0006F000000EFD0DFC96F00400597E70100CF
:10290000938747CA03A7070097E701009387C7CAC1
:1029100083A70700631AF70097E70100938747AC86
:1029200023A007006F008002EF0090286F000002D4
:1029300097E70100938707C983A70700638807000B
:10294000EF109051EF105019EF10105513000000C8
:102950008320C1021301010367800000130101FEFF
:102960002326A100232E01008327C100232CF10080
:102970008327C10063960700737004306F00000066
:102980008327810103A7470197E70100938787C148
:102990006316F700930710006F0080009307000094
:1029A000638E07028327810103A7870297E701004F
:1029B000938787BC6304F7028327810183A787027B
:1029C00063960700930710006F00800093070000D4
:1029D0006386070093071000232EF1008327C101AF
:1029E000138507001301010267800000130101FD38
:1029F000232611022326A1008327C100232EF100E4
:102A00008327C10063960700737004306F000000D5
:102A10008327C1016384070C97E701009387479CD4
:102A200083A707000327C101630AF70AEF10D0420A
:102A30000325C101EFF09FF2130705009307100073
:102A4000631CF7088327C10193874700138507009C
:102A5000EFD01FF48327C10103A7C70297E7010046
:102A6000938707B683A7070063FCE7008327C101AC
:102A700003A7C70297E70100938787B423A0E70065
:102A80008327C10103A7C702930707009397270075
:102A9000B387E7009397270017E701001307479EC6
:102AA0003387E7008327C101938747009385070099
:102AB00013050700EFD09FD98327C10103A7C702E1
:102AC00097E701009387C79183A7070083A7C702F1
:102AD0006364F700EFD0DFABEF10103C1300000091
:102AE0008320C1021301010367800000130101FD6F
:102AF000232611022326A100232E01008327C100D3
:102B0000232CF1008327C100639607007370043003
:102B10006F000000EFD01FBF93070500232AF100CC
:102B200003258101EFF09FE31307050093071000D1
:102B30006314F70C97E70100938747AA83A7070060
:102B40006390070A8327810103A7C70297E7010063
:102B50009387078983A7070083A7C7026366F700E7
:102B600093071000232EF1008327810193874700EC
:102B700013850700EFD0DFE18327810103A7C70298
:102B800097E701009387C7A383A7070063FCE700CB
:102B90008327810103A7C70297E70100938747A214
:102BA00023A0E7008327810103A7C702930707003B
:102BB00093972700B387E7009397270017E7010053
:102BC0001307078C3387E70083278101938747002A
:102BD0009385070013050700EFD05FC76F00C001A2
:102BE00083278101938787019385070017E50100FB
:102BF00013058598EFD09FC58327410113850700F2
:102C0000EFD09FAE8327C101138507008320C10247
:102C10001301010367800000130101FE232E110040
:102C2000930800001308000093070000130700003A
:102C3000930600001306004097D501009385853C5C
:102C400017150000130505FBEFF08FAF2326A10039
:102C50000327C100930710006316F700EF20C03A66
:102C60002326A1000327C10093071000631EF7026B
:102C70007370043097E70100938707961307F0FFFE
:102C800023A0E70097E701009387C793130710007D
:102C900023A0E70097E701009387479223A007004E
:102CA000EFD04FF46F0040018327C1006396070007
:102CB000737004306F000000130000008320C10116
:102CC0001301010267800000130101FF2326110098
:102CD0007370043097E701009387C78E23A0070025
:102CE000EFD09F82130000008320C1001301010177
:102CF0006780000097E701009387478E83A707004E
:102D00001387170097E701009387478D23A0E700FB
:102D10001300000067800000130101FE232E110044
:102D20002326010097E701009387478B83A70700BD
:102D300063960700737004306F000000EF10D0112D
:102D400097E701009387878983A707001387F7FF19
:102D500097E701009387878823A0E70097E70100A2
:102D60009387C78783A707006394071697E7010037
:102D70009387878483A70700638C07146F00800CF8
:102D800097D701009387477F83A7C70083A7C70012
:102D90002324F1008327810093878701138507008F
:102DA000EFD01FBF8327810093874700138507005B
:102DB000EFD01FBE8327810003A7C70297E701005A
:102DC0009387078083A7070063FCE70083278100C0
:102DD00003A7C70297D701009387877E23A0E70048
:102DE0008327810003A7C702930707009397270053
:102DF000B387E7009397270017D7010013074768A9
:102E00003387E70083278100938747009385070076
:102E100013050700EFD09FA38327810003A7C702F4
:102E200097D701009387C75B83A7070083A7C702D3
:102E3000636AF70097D7010093874779130710005B
:102E400023A0E70097D701009387077383A70700A4
:102E5000E39807F297D701009387077783A70700C6
:102E6000638807046F00C003EF00002B9307050081
:102E7000638A070097D701009387477513071000EF
:102E800023A0E70097D701009387077483A7070063
:102E90001387F7FF97D701009387077323A0E700F5
:102EA00097D701009387477283A70700E39E07FA2D
:102EB00097D701009387877103A707009307100036
:102EC0006318F700930710002326F100EFD04FECB2
:102ED000EF10807C8327C100138507008320C10188
:102EE0001301010267800000130101FE232E11006F
:102EF000EF10807697D701009387476C83A7070070
:102F00002326F100EF1040798327C10013850700C5
:102F10008320C1011301010267800000130101FE3B
:102F2000232E1100EFD00FFE930705002326F1009A
:102F300097D701009387876883A707002324F100B0
:102F40008327C10013850700EFD00FFA8327810084
:102F5000138507008320C10113010102678000006F
:102F600097D701009387476583A70700138507005C
:102F700067800000130101FD232611022326A10012
:102F80002324B1002322C100232E01009307A000B7
:102F9000232CF100EFF01FD697D701009387C7616C
:102FA00083A7070003278100636CF714832781013F
:102FB0009387F7FF232CF1008327C10193975700D4
:102FC0000327C100B306F700032781019307070019
:102FD00093972700B387E7009397270017D701003F
:102FE0001307074AB387E70013061000938507000D
:102FF00013850600EF108004130705008327C10125
:10300000B387E700232EF10083278101E39007FABD
:103010008327C101939757000327C1003307F700A7
:1030200097D701009387C75483A707001306200092
:103030009385070013050700EF10400013070500F4
:103040008327C101B387E700232EF1008327C10145
:10305000939757000327C1003307F70097D7010064
:103060009387475183A70700130620009385070025
:1030700013050700EF00907C130705008327C101AB
:10308000B387E700232EF1008327C10193975700F0
:103090000327C100B307F7001306400097D50100CE
:1030A0009385C54E13850700EF005079130705007F
:1030B0008327C101B387E700232EF1008327C101D5
:1030C000939757000327C100B307F700130630009A
:1030D00097D501009385054D13850700EF00107605
:1030E000130705008327C101B387E700232EF100F2
:1030F00083274100638607008327410023A0070040
:10310000EFF09FC18327C101138507008320C1020F
:103110001301010367800000130101FD2326110242
:10312000232E010097D701009387474B83A7070001
:10313000639C072297D701009387474883A707001E
:103140001387170097D701009387474723A0E7000D
:1031500097D701009387874683A70700232CF100A8
:1031600083278101639C070697D701009387474017
:1031700083A7070083A707006386070073700430E6
:103180006F00000097D701009387873E83A7070051
:10319000232AF10097D701009387C73D03A70700B3
:1031A00097D701009387C73C23A0E70097D701007A
:1031B0009387473C0327410123A0E70097D70100ED
:1031C0009387074183A707001387170097D701004C
:1031D0009387074023A0E700EF10001097D7010066
:1031E0009387873F83A7070003278101636CF7124A
:1031F00097D701009387C73783A7070083A70700E6
:1032000063960700930710006F008000930700008B
:10321000638C070097D701009387073C1307F0FFE3
:1032200023A0E7006F00001097D701009387473471
:1032300083A7070083A7C70083A7C7002328F1003F
:103240008327010183A747002326F100032781017B
:103250008327C100637CF70097D701009387C737A6
:103260000327C10023A0E7006F00C00B83270101E3
:103270009387470013850700EFD08FF18327010163
:1032800083A78702638A0700832701019387870149
:1032900013850700EFD0CFEF8327010103A7C702F3
:1032A00097D701009387C73183A7070063FCE70026
:1032B0008327010103A7C70297D7010093874730EF
:1032C00023A0E7008327010103A7C7029307070094
:1032D00093972700B387E7009397270017D701003C
:1032E0001307071A3387E7008327010193874700F5
:1032F0009385070013050700EFD04FD58327010101
:1033000003A7C70297D701009387870D83A70700FC
:1033100083A7C702E36EF7EC93071000232EF1009A
:103320006FF01FED97D701009387870B83A70700E6
:1033300003A7C70297D60100938686149307070058
:1033400093972700B387E70093972700B387F6008A
:1033500003A707009307100063F6E7029307100026
:10336000232EF1006F00000297D701009387C72535
:1033700083A707001387170097D701009387C724F7
:1033800023A0E70097D701009387472483A707006E
:103390006386070093071000232EF1008327C101E5
:1033A000138507008320C102130101036780000019
:1033B000130101FE232E110097D7010093870722E6
:1033C00083A70700638C070097D701009387072026
:1033D0001307100023A0E7006F00C01897D7010063
:1033E0009387C71E23A0070097D70100938747FF45
:1033F00083A7070083A707032326F100B7A7A5A586
:103400009387575A2324F1008327C10083A707001D
:10341000032781006310F7048327C10093874700C7
:1034200083A70700032781006316F7028327C100E3
:103430009387870083A7070003278100631CF70099
:103440008327C1009387C70083A707000327810054
:103450006302F70697D70100938787F803A7070051
:1034600097D701009387C7F783A707009387470380
:103470009385070013050700EF40C03D6F008003F0
:1034800097D701009387C71383A7070063960700A8
:10349000737004306F00000097D7010093874712C4
:1034A00083A707001387F7FF97D70100938747117A
:1034B00023A0E70097D701009387871003A7070091
:1034C00097D601009386C6FB9307070093972700C2
:1034D000B387E70093972700B387F60083A7070019
:1034E000E38007FA97D701009387870D03A70700AA
:1034F0009307070093972700B387E7009397270068
:1035000017D701001307C7F7B387E7002322F1009D
:103510008327410083A7470003A747008327410073
:1035200023A2E7008327410003A747008327410028
:1035300093878700631CF7008327410083A7470018
:1035400003A747008327410023A2E7008327410008
:1035500083A7470003A7C70097D70100938747E8D1
:1035600023A0E700130000008320C1011301010222
:1035700067800000130101FD232611022326A1000C
:103580002324B1008327C1006396070073700430C1
:103590006F00000097D70100938787E483A7070097
:1035A00093878701938507000325C100EFD0CFB132
:1035B00097D701009387C7E283A707009387470047
:1035C00013850700EFD0CFBC032781009307F0FFDE
:1035D0006314F70297D70100938787E083A707005A
:1035E000938747009385070017D50100130585FBD6
:1035F000EFD0CFA56F00400297D70100938707FC5B
:1036000083A7070003278100B307F700232EF100EB
:103610000325C101EF00900B130000008320C102BD
:103620001301010367800000130101FD232611022D
:103630002326A1002324B1002322C1008327C10037
:1036400063960700737004306F00000097D7010085
:103650009387C7F883A70700639607007370043049
:103660006F00000097D70100938787D783A70700D3
:10367000832681003707008033E7E60023ACE700AC
:1036800097D701009387C7D583A707009387870142
:10369000938507000325C100EFD04F9B97D701000A
:1036A000938707D483A707009387470013850700F4
:1036B000EFD00FAE032741009307F0FF6314F7022A
:1036C00097D701009387C7D183A707009387470047
:1036D0009385070017D501001305C5ECEFD00F97B0
:1036E0006F00400297D70100938747ED83A707003B
:1036F00003274100B307F700232EF1000325C10182
:10370000EF00C07C130000008320C10213010103FD
:1037100067800000130101FD232611022326A1006A
:103720002324B1002322C1008327C1006396070030
:10373000737004306F00000097D70100938747CA69
:1037400083A7070093878701938507000325C1009E
:10375000EFD0CF8F97D70100938787C883A7070043
:103760009387470013850700EFD08FA203274100FE
:10377000930710006314F70297D70100938747C699
:1037800083A70700938747009385070017D501009B
:10379000130545E1EFD08F8B6F00400297D70100F2
:1037A0009387C7E183A7070003278100B307F700CA
:1037B000232EF1000325C101EF004071130000002A
:1037C0008320C1021301010367800000130101FD82
:1037D000232611022326A1008327C10083A7C70047
:1037E00083A7C700232CF10083278101639607007C
:1037F000737004306F000000832781019387870175
:1038000013850700EFD0CF9897D70100938707DD86
:1038100083A70700639E07068327810193874700DC
:1038200013850700EFD0CF968327810103A7C70236
:1038300097D701009387C7D883A7070063FCE700E9
:103840008327810103A7C70297D70100938747D732
:1038500023A0E7008327810103A7C702930707007E
:1038600093972700B387E7009397270017D70100A6
:10387000130707C13387E700832781019387470038
:103880009385070013050700EFC05FFC6F00C001C0
:1038900083278101938787019385070017D501004E
:1038A000130585CDEFC09FFA8327810103A7C702C7
:1038B00097D701009387C7B283A7070083A7C702E2
:1038C00063F0E70293071000232EF10097D7010061
:1038D0009387C7CF1307100023A0E7006F00800075
:1038E000232E01008327C101138507008320C10215
:1038F0001301010367800000130101FD232611025B
:103900002326A1002324B10097D70100938707CD78
:1039100083A7070063960700737004306F000000F0
:1039200003278100B70700803367F7008327C100B2
:1039300023A0E7008327C10083A7C700232CF10041
:103940008327810163960700737004306F000000C5
:103950000325C100EFD0CF838327810193874700E0
:1039600013850700EFD0CF828327810103A7C70209
:1039700097D701009387C7C483A7070063FCE700BC
:103980008327810103A7C70297D70100938747C305
:1039900023A0E7008327810103A7C702930707003D
:1039A00093972700B387E7009397270017D7010065
:1039B000130707AD3387E70083278101938747000B
:1039C0009385070013050700EFC05FE88327810197
:1039D00003A7C70297D70100938787A083A7070093
:1039E00083A7C70263F0E70293071000232EF100BC
:1039F00097D70100938787BD1307100023A0E70026
:103A00006F008000232E01008327C101138507006A
:103A10008320C1021301010367800000130101FF2D
:103A20002326A1008327C10063960700737004302A
:103A30006F00000097D70100938787B903A707009D
:103A40008327C10023A0E70097D70100938707B71A
:103A500003A707008327C10023A2E700130000008B
:103A60001301010167800000130101FD23261102EB
:103A70002326A1002324B1008327C10063960700F9
:103A8000737004306F000000832781006396070085
:103A9000737004306F000000EF00103C97D70100F6
:103AA0009387C7B183A70700232CF10083278100E8
:103AB00003A707009307F0FF6316F700232E01000A
:103AC0006F0000098327C10003A7070097D70100F3
:103AD000938707B083A707006300F7028327C1001D
:103AE00083A74700032781016368F700930710004D
:103AF000232EF1006F00C0058327C10083A7470074
:103B0000032781013307F7408327810083A707003C
:103B1000637CF7028327810003A707008327C10086
:103B200083A6470083278101B387F6403307F70058
:103B30008327810023A0E7000325C100EFF01FEEDB
:103B4000232E01006F00C00093071000232EF10008
:103B5000EF0090348327C101138507008320C10241
:103B6000130101036780000097D70100938707A620
:103B70001307100023A0E700130000006780000077
:103B8000130101FE2326A1008327C100638E0700D5
:103B90008327C100232CF1008327810183A7C70459
:103BA000232EF1006F008000232E01008327C10126
:103BB000138507001301010267800000130101FE55
:103BC0002326A1002324B1008327C100638C0700B2
:103BD0008327C100232EF1008327C1010327810021
:103BE00023A6E70413000000130101026780000010
:103BF000130101FE232E11002326A100EF00002156
:103C000097D701009387C78703A707009307100082
:103C1000E3F6E7FEEFC0DF976FF05FFE130101FCF4
:103C2000232E1102232EA100232CB100232AC10030
:103C30002328D100930707002317F1002326010250
:103C40006F004004032781018327C102B307F700F7
:103C500003C707008326C1018327C102B387F6008B
:103C6000238AE702032781018327C102B307F700F4
:103C700083C70700638007028327C1029387170069
:103C80002326F1020327C1029307F000E3FCE7FAC1
:103C90006F008000130000008327C101A381070487
:103CA000032741019307900063F6E7009307900014
:103CB000232AF1008327C1010327410123A6E7023C
:103CC0008327C1010327410123A8E7048327C101FA
:103CD00023AA07048327C1019387470013850700A0
:103CE000EFC01FB58327C1019387870113850700A4
:103CF000EFC01FB48327C1010327C10123A8E70038
:103D00001307A000832741013307F7408327C10130
:103D100023ACE7008327C1010327C10123A2E702E7
:103D20008327C10123A207048327C10123AC070411
:103D30008327C10123AE0704130000008320C103C1
:103D40001301010467800000130101FE232E1100FE
:103D5000232601006F0080030327C100930707009B
:103D600093972700B387E7009397270017C70100B1
:103D700013070771B387E70013850700EFC0DFA5BE
:103D80008327C100938717002326F1000327C10072
:103D900093079000E3F2E7FC17C501001305C57A0D
:103DA000EFC09FA317C501001305457BEFC0DFA23D
:103DB00017C501001305457CEFC01FA217C5010000
:103DC0001305C57CEFC05FA117C501001305857DF4
:103DD000EFC09FA097C701009387877917C701009D
:103DE0001307877623A0E70097C70100938787789A
:103DF00017C701001307877623A0E7001300000010
:103E00008320C1011301010267800000130101FE3C
:103E1000232E11006F008009EFE0DFED97C701004E
:103E20009387C77683A7070093B7170093F7F70F19
:103E30002326F100EFE05FEE8327C10063980706B9
:103E4000EF00900197C701009387477483A7C700CD
:103E500083A7C7002324F1008327810093874700AD
:103E600013850700EFC0DFB297C701009387C774BF
:103E700083A707001387F7FF97C701009387C773CE
:103E800023A0E70097C701009387877183A70700E6
:103E90001387F7FF97C701009387877023A0E70078
:103EA000EF00807F03258100EF00C03F97C701002E
:103EB0009387076F83A70700E39007F613000000BE
:103EC0008320C1011301010267800000130101FE7C
:103ED000232E11002326A10097C701009387475086
:103EE00083A707000327C10023A2E70097C70100AB
:103EF0009387C76C83A707000327C1006378F70285
:103F000097C701009387076703A7070097C70100BA
:103F10009387074D83A70700938747009385070082
:103F200013050700EFC05F9A6F00000597C70100F7
:103F30009387076403A7070097C701009387474A41
:103F400083A70700938747009385070013050700A1
:103F5000EFC09F9797C701009387076883A7070063
:103F60000327C100637AF70097C701009387C766EC
:103F70000327C10023A0E700130000008320C10134
:103F80001301010267800000130101FD23261102C5
:103F9000930705002324B1002317F1008327810034
:103FA000639E07008357E10093972700138507005E
:103FB000EF20804B930705006F008000832781006E
:103FC000232CF10083278101638A07021305000671
:103FD000EF208049232EA1008327C101638A0700B7
:103FE0008327C1010327810123A8E7026F00400155
:103FF00003258101EF2000676F008000232E010060
:104000008327C101638207028327C10103A7070336
:104010008357E10093972700138607009305500A02
:1040200013050700EF20D0068327C1011385070081
:104030008320C1021301010367800000130101FC0A
:10404000232E1102232C81022326A1002324B10058
:104050002322C100232601028327810083A70700B2
:104060006388071C832781002324F10283278102B0
:1040700083A7470003A747008327810223A2E70005
:104080008327810203A74700832781029387870044
:10409000631CF7008327810283A7470003A747001B
:1040A0008327810223A2E7008327810283A7470099
:1040B00083A7C7002322F102832781002320F10276
:1040C0008327010283A7470003A747008327010234
:1040D00023A2E7008327010203A7470083270102E9
:1040E00093878700631CF7008327010283A747009B
:1040F00003A747008327010223A2E70083270102C9
:1041000083A7470083A7C700232EF1008327C1029E
:10411000939757000327C100B307F7000327C10196
:1041200023A0E7008327C102939757000327C1000C
:10413000B307F7000327C1011307470323A2E700D2
:104140008327C102939757000327C100B307F700E5
:104150000327C1010327870423A4E7008327C102A3
:10416000939757000327C100B307F70003274100C7
:1041700023A6E7008327C102939757000327C100B6
:10418000B307F7000327C1010327C70223A8E700ED
:1041900003274100930730006314F7028327C1010E
:1041A00083A78702638E07008327C1029397570076
:1041B0000327C100B307F7001307200023A6E70079
:1041C0008327C102939757000327C100B307F70065
:1041D0000327C1010327070523AAE7008327C1029C
:1041E000939757000327C100B307F70023AC0700DC
:1041F0008327C10183A607038327C1029397570032
:104200000327C1003304F70013850600EF00C00345
:1042100093070500231EF4008327C102938717002C
:104220002326F1020327C10183274102E316F7E8A1
:104230008327C102138507008320C1030324810360
:104240001301010467800000130101FE2326A10071
:10425000232E01006F00C0018327C1009387170040
:104260002326F1008327C10193871700232EF10035
:104270008327C10003C707009307500AE30EF7FC2A
:104280008327C10193D72700232EF1008327C10183
:104290009397070193D707011385070013010102C4
:1042A00067800000130101FE232E11002326A100C8
:1042B0008327C10083A7070313850700EF20803AF7
:1042C0000325C100EF20003A130000008320C10144
:1042D0001301010267800000130101FF97C701006D
:1042E0009387072983A7070083A707006396070022
:1042F000930710006F00800093070000638C070095
:1043000097C701009387472D1307F0FF23A0E7000D
:104310006F00000397C701009387872583A70700D5
:1043200083A7C70083A7C7002326F1008327C10006
:1043300003A7470097C701009387072A23A0E70038
:10434000130000001301010167800000130101FF49
:1043500097C701009387C70883A707002326F100AA
:104360008327C10013850700130101016780000046
:10437000130101FF97C701009387C72483A7070094
:1043800063980700930710002326F1006F00400296
:1043900097C701009387872483A7070063980700C6
:1043A000930720002326F1006F00800023260100E0
:1043B0008327C100138507001301010167800000F6
:1043C000130101FD232611022326A1008327C1002A
:1043D000232EF1008327C100638A07128327C101BE
:1043E00003A7C70297C70100938787FF83A707002A
:1043F00083A7C702637CF7108327C10183A78701C6
:1044000063C2070297C70100938787FD83A7070050
:1044100083A7C7021307A0003307F7408327C10112
:1044200023ACE7008327C10183A647018327C1018D
:1044300003A7C7029307070093972700B387E700F6
:104440009397270017C7010013078703B387E70077
:104450006396F600930710006F008000930700003A
:10446000638A07088327C1019387470013850700E4
:10447000EFC00FD297C70100938787F683A7070085
:1044800003A7C7028327C10123A6E7028327C1012F
:1044900003A7C70297C701009387871283A7070066
:1044A00063FCE7008327C10103A7C70297C7010088
:1044B0009387071123A0E7008327C10103A7C70241
:1044C0009307070093972700B387E7009397270088
:1044D00017C701001307C7FA3387E7008327C10115
:1044E000938747009385070013050700EFC00FB6B9
:1044F0006F00C00197C70100938787EE83A707006D
:1045000003A7C7028327C10123A6E7021300000007
:104510008320C1021301010367800000130101FD24
:10452000232611022326A1008327C100232CF1009A
:10453000232E01008327C1006386071097C701005F
:10454000938707EA83A70700032781016306F70023
:10455000737004306F0000008327810183A7470533
:1045600063960700737004306F0000008327810199
:1045700083A747051387F7FF8327810123AAE70451
:104580008327810103A7C7028327810183A707052A
:10459000630AF70A8327810183A747056394070A03
:1045A000832781019387470013850700EFC04FBE23
:1045B0008327810103A707058327810123A6E7023B
:1045C0008327810183A7C7021307A0003307F740A1
:1045D0008327810123ACE7008327810103A7C7025A
:1045E00097C701009387C7FD83A7070063FCE70017
:1045F0008327810103A7C70297C70100938747FC60
:1046000023A0E7008327810103A7C70293070700C0
:1046100093972700B387E7009397270017C70100F8
:10462000130707E63387E700832781019387470055
:104630009385070013050700EFC04FA193071000F3
:10464000232EF1008327C101138507008320C102B7
:1046500013010103678000007370043097C70100E5
:10466000938747F683A707006384070297C7010073
:10467000938707D783A7070003A7470413071700EB
:1046800023A2E70497C70100938787D583A7070074
:10469000130000006780000097C70100938787F22E
:1046A00083A707006384070497C70100938747D354
:1046B00083A7070083A74704638A070297C70100FF
:1046C000938707D283A7070003A747041307F7FFC1
:1046D00023A2E70497C70100938787D083A7070029
:1046E00083A747046394070073600430130000003D
:1046F00067800000130101FF97C70100938747CE31
:1047000083A7070083A787012326F10097C701002D
:10471000938707CD83A7070003A7C70297C70100A8
:10472000938707CC83A707009306A0003387E64052
:1047300023ACE7008327C1001385070013010101A3
:104740006780000097C70100938787C983A7070088
:10475000638E070097C70100938787C883A7070068
:1047600003A747051307170023AAE70497C701000B
:10477000938707C783A7070013850700678000009A
:10478000130101FD232611022326A1002324B100D9
:10479000EFF09FEC97C70100938787C483A70700BA
:1047A00083A787056396070897C70100938747C3C8
:1047B00083A707001307100023AEE70483278100B7
:1047C0006388070697C70100938787C183A70700FF
:1047D0009387470013850700EFC08F9B0327810055
:1047E0009307F0FF6314F70297C70100938747BF51
:1047F00083A70700938747009385070017C501002B
:10480000130545DAEFC08F846F00400297C701009F
:104810009387C7DA83A7070003278100B307F70050
:10482000232EF1000325C101EFF04FEAEFB05FD670
:10483000EFF09FE6EFF05FE297C70100938747BA7A
:1048400083A7070083A78705232CF1008327810115
:10485000638C07028327C100638C070097C70100A0
:10486000938707B883A7070023AC07046F00C00134
:1048700097C701009387C7B683A7070003A78705DB
:104880001307F7FF23ACE70497C70100938747B5E9
:1048900083A7070023AE0704EFF01FE08327810101
:1048A000138507008320C102130101036780000004
:1048B000130101FD232611022326A1002324B100A8
:1048C0002322C1002320D100EFF01FD997C7010098
:1048D000938707B183A7070003A7C70593072000A5
:1048E0006306F70A97C70100938787AF83A707007E
:1048F00083A687050327C1001347F7FF33F7E600B8
:1049000023ACE70497C70100938787AD83A707000F
:104910001307100023AEE70483270100638807060E
:1049200097C701009387C7AB83A70700938747000A
:1049300013850700EFC0CF85032701009307F0FF21
:104940006314F70297C70100938787A983A707001D
:10495000938747009385070017C50100130585C499
:10496000EFB0DFEE6F00400297C70100938707C5E5
:1049700083A7070003270100B307F700232CF100EA
:1049800003258101EFF08FD4EFB09FC0EFF0DFD0AF
:10499000EFF09FCC83274100638E070097C701008B
:1049A000938707A483A7070003A7870583274100F0
:1049B00023A0E70097C70100938787A283A707007A
:1049C00003A7C705930710006316F700232E010005
:1049D0006F00C00297C70100938787A083A70700D5
:1049E00083A68705032781001347F7FF33F7E60007
:1049F00023ACE70493071000232EF10097C70100B2
:104A00009387079E83A7070023AE0704EFF0DFC854
:104A10008327C101138507008320C102130101030D
:104A200067800000130101FD232611022326A10047
:104A30002324B1002322C1002320D10093071000BA
:104A4000232EF1008327C1006396070073700430A2
:104A50006F0000008327C100232CF100EFF0DFBFBF
:104A600083270100638A07008327810103A7870545
:104A70008327010023A0E7008327810183A7C705BF
:104A8000232AF100832781011307200023AEE704C6
:104A9000032741009307400063ECE70883274100A8
:104AA0001397270097B7010093874756B307F7007E
:104AB00003A7070097B7010093874755B307F7008F
:104AC000678007008327810103A78705832781006B
:104AD0003367F7008327810123ACE7046F004005AB
:104AE0008327810183A78705138717008327810107
:104AF00023ACE7046F00C0038327810103278100F3
:104B000023ACE7046F00C002032741019307200094
:104B1000630AF700832781010327810023ACE704A0
:104B20006F000001232E01006F00800013000000C1
:104B300003274101930710006316F70A83278101B9
:104B40009387470013850700EFB09FE48327810117
:104B500003A7C70297C70100938787A683A707000B
:104B600063FCE7008327810103A7C70297C7010001
:104B7000938707A523A0E7008327810103A7C70226
:104B80009307070093972700B387E70093972700C1
:104B900017C701001307C78E3387E70083278101FA
:104BA000938747009385070013050700EFB01FCADE
:104BB0008327810183A7870263860700737004300F
:104BC0006F0000008327810103A7C70297C7010078
:104BD0009387078183A7070083A7C70263F4E700D1
:104BE000EFB01F9BEFF05FAB8327C1011385070078
:104BF0008320C1021301010367800000130101FC3F
:104C0000232E1102232EA100232CB100232AC10040
:104C10002328D1002326E100930710002326F10268
:104C20008327C10163960700737004306F00000092
:104C30008327C1012324F102EFB0DFAC9307050005
:104C40002322F10283270101638A0700832781025F
:104C500003A787058327010123A0E700832781029B
:104C600083A7C7052320F1028327810213072000B1
:104C700023AEE704032741019307400063ECE708F4
:104C8000832741011397270097B70100938747397E
:104C9000B307F70003A7070097B7010093874738CA
:104CA000B307F700678007008327810203A7870502
:104CB000832781013367F7008327810223ACE70450
:104CC0006F0040058327810283A78705138717009C
:104CD0008327810223ACE7046F00C003832781028E
:104CE0000327810123ACE7046F00C0020327010200
:104CF00093072000630AF7008327810203278101BD
:104D000023ACE7046F000001232601026F0080003E
:104D10001300000003270102930710006314F70E2D
:104D20008327810283A7870263860700737004309C
:104D30006F00000097C701009387478A83A7070089
:104D4000639E070683278102938747001385070028
:104D5000EFB01FC48327810203A7C70297C70100D2
:104D60009387078683A7070063FCE70083278102F8
:104D700003A7C70297C701009387878423A0E70092
:104D80008327810203A7C702930707009397270091
:104D9000B387E7009397270017B701001307476E03
:104DA0003387E700832781029387470093850700B5
:104DB00013050700EFB09FA96F00C0018327810290
:104DC000938787019385070017B501001305C57AFE
:104DD000EFB0DFA78327810203A7C70297B70100BF
:104DE0009387076083A7070083A7C70263FCE700D8
:104DF0008327C100638807008327C10013071000C1
:104E000023A0E7008327410213850700EFB0DF8D61
:104E10008327C102138507008320C1031301010406
:104E200067800000130101FD232611022326A10043
:104E30002324B1008327C1006396070073700430F8
:104E40006F0000008327C100232EF100EFB09F8B7D
:104E500093070500232CF1008327C10183A7C70511
:104E6000232AF1008327C1011307200023AEE704A2
:104E70008327C10183A78705138717008327C101F3
:104E800023ACE70403274101930710006314F70ED6
:104E90008327C10183A787026386070073700430EC
:104EA0006F00000097B701009387477383A707003F
:104EB000639E07068327C101938747001385070078
:104EC000EFB01FAD8327C10103A7C70297B7010049
:104ED0009387076F83A7070063FCE7008327C1015F
:104EE00003A7C70297B701009387876D23A0E70048
:104EF0008327C10103A7C7029307070093972700E1
:104F0000B387E7009397270017B7010013074757A8
:104F10003387E7008327C101938747009385070004
:104F200013050700EFB09F926F00C0018327C101F6
:104F3000938787019385070017B501001305C563A3
:104F4000EFB0DF908327C10103A7C70297B7010025
:104F50009387074983A7070083A7C70263FCE7007D
:104F600083278100638807008327810013071000CF
:104F700023A0E7008327810113850700EFB0CFF658
:104F8000130000008320C1021301010367800000A9
:104F9000130101FD232611022326A1008327C1004E
:104FA000232CF10083278101639A070097B7010042
:104FB0009387074383A707006F0080008327810141
:104FC000232CF100EFF04FE98327810103A7C705E8
:104FD00093072000631CF7008327810123AE070499
:104FE00093071000232EF1006F008000232E010094
:104FF000EFF08FEA8327C101138507008320C102E8
:105000001301010367800000130101FE232E11002C
:1050100023260100EF00D00F97B701009387475F69
:1050200083A70700638A07029308000013080000A3
:1050300093070000130720009306000013060040AA
:1050400097B50100938505FF170500001305852E10
:10505000EFC01FEF2326A1008327C100639607003E
:10506000737004306F0000008327C10013850700B0
:105070008320C1011301010267800000130101FCBC
:10508000232E1102232EA100232CB100232AC100BC
:105090002328D1002326E10083278101639607009E
:1050A000232601026F0080061305C002EF10C03BEB
:1050B0002326A1028327C102638A0704EF0050055B
:1050C0008327C1020327C10123A0E7008327C10270
:1050D0000327810123ACE7008327C1020327410195
:1050E00023AEE7008327C1020327010123A0E702C3
:1050F0008327C1020327C10023A2E7028327C1023D
:105100009387470013850700EFB08FF28327810153
:1051100063960700737004306F0000008327C1029C
:10512000138507008320C103130101046780000079
:10513000130101FB23261104232EA100232CB1000F
:10514000232AC1002328D1002326E100232E0102B7
:105150008327C10163960700737004306F0000005D
:1051600097B701009387C74A83A70700638C070A94
:10517000832781012326F102832741012328F1029D
:105180008327C101232AF1020327810193075000DD
:1051900063C6E706EFF0CF9D1307050093072000D5
:1051A0006318F70297B701009387874683A7070024
:1051B0001307C102930600000326C10093050700F0
:1051C00013850700EFB01FD2232EA1026F008005C8
:1051D00097B701009387C74383A707001307C1024E
:1051E00093060000130600009305070013850700CF
:1051F000EFB05FCF232EA1026F00C00297B701006E
:105200009387074183A707001307C1029306000095
:10521000032601019305070013850700EFB09FF0F7
:10522000232EA1028327C103138507008320C10415
:105230001301010567800000130101FE2326A10070
:105240008327C100232EF1008327C1006396070046
:10525000737004306F0000008327C10183A707002B
:10526000138507001301010267800000130101FD8F
:10527000232611022326A1002324B10097B70100A1
:105280009387873883A7070083A7C70083A7C70032
:10529000232EF1008327C101938747001385070060
:1052A000EFB00FEF8327C10103A7C70193071000D9
:1052B0006310F7068327C10103A787018327C10075
:1052C000B307F7008326C1000326810093850700FA
:1052D0000325C101EF00802213070500930710008A
:1052E0006318F70213070000930600000326C100AD
:1052F000930500000325C101EFF09FE3232CA100DB
:105300008327810163960700737004306F000000EB
:105310008327C10183A747020325C101E780070056
:10532000130000008320C102130101036780000005
:10533000130101FD232611022326A10093078101F9
:1053400013850700EF00800E232EA1008327810123
:10535000938507000325C101EF00C000EF0000287E
:105360006FF0DFFD130101FD232611022326A100AA
:105370002324B100EFD01F98930781011385070004
:10538000EF004011232EA1008327810163960708B7
:1053900083278100639207020327C1008327C1018D
:1053A00063ECE700EFD05F978325C1010325C100BF
:1053B000EFF0DFEB6F008006832781006380070238
:1053C00097B701009387872483A7070083A7070067
:1053D00093B7170093F7F70F2324F10097B7010055
:1053E0009387072383A607000327C1008327C101F2
:1053F000B307F74003268100938507001385060055
:10540000EFC01FABEFD05F919307050063980700D3
:10541000EFB00F986F008000EFD01F9013000000D6
:105420008320C1021301010367800000130101FE04
:105430002326A10097B701009387071D83A70700C4
:1054400083A7070093B7170093F7F70F1387070099
:105450008327C10023A0E7008327C10083A707009B
:105460006390070297B701009387071A83A7070085
:1054700083A7C70083A70700232EF1006F008000D9
:10548000232E01008327C1011385070013010102A8
:1054900067800000130101FD232611022326A100CD
:1054A000EFD09FA4232EA10097B701009387871602
:1054B00083A707000327C101637CF700EF0040309A
:1054C0008327C1001307100023A0E7006F00C0006E
:1054D0008327C10023A0070097B701009387871394
:1054E0000327C10123A0E7008327C101138507001B
:1054F0008320C1021301010367800000130101FD35
:10550000232611022326A1002324B1002322C10057
:105510002320D100232E01008327C100032781000F
:1055200023A2E7008327C1000327C10023A8E700C7
:10553000032781008327410063E6E7040327410036
:10554000832701003307F7408327C10083A7870122
:105550006368F70093071000232EF1006F00C00668
:1055600097B701009387870A03A707008327C10025
:10557000938747009385070013050700EFB0CFB46A
:105580006F0080040327410083270100637EF7003A
:1055900003278100832701006368F7009307100049
:1055A000232EF1006F00400297B701009387C705D3
:1055B00003A707008327C10093874700938507004F
:1055C00013050700EFB04FB08327C1011385070013
:1055D0008320C1021301010367800000130101FC55
:1055E000232E11026F00001A8327010163D20704E2
:1055F00093070101938747002326F1028327C10205
:1056000063960700737004306F0000008327C102A7
:1056100083A607008327C10203A747008327C1028F
:1056200083A787009385070013050700E78006001E
:105630008327010163C60714832781012324F10214
:105640008327810283A74701638A0700832781029A
:105650009387470013850700EFB08FB39307C1000E
:1056600013850700EFF01FE32322A1028327010126
:10567000130790006368F7101397270097B701008E
:105680009387C79BB307F70003A7070097B70100ED
:105690009387C79AB307F700678007000327410184
:1056A0008327810283A78701B307F70003274101FE
:1056B0009306070003264102938507000325810214
:1056C000EFF0DFE31307050093071000631CF70AF0
:1056D0008327810283A7470203258102E780070011
:1056E0008327810203A7C70193071000631CF708F3
:1056F000032741018327810283A78701B307F700AE
:1057000013070000930600001386070093050000AE
:1057100003258102EFF0DFA12320A10283270102EC
:1057200063920706737004306F0000000327410185
:105730008327810223ACE7008327810283A78701A7
:1057400063960700737004306F00000083278102A6
:1057500003A7870183274102B307F700832641028D
:10576000032641029385070003258102EFF01FD92C
:105770006F00400103258102EF00D06E6F008000B2
:105780001300000097B70100938787E883A70700FD
:10579000130701019306000013060000930507009C
:1057A00013850700EFB0DFC093070500E39E07E213
:1057B000130000008320C10313010104678000006F
:1057C000130101FD232611026F00C00E97B70100DF
:1057D000938787E383A7070083A7C70083A70700F2
:1057E000232CF10097B70100938707E283A70700F6
:1057F00083A7C70083A7C700232AF100832741019D
:105800009387470013850700EFB08F9883274101E6
:1058100083A7470203254101E78007008327410151
:1058200003A7C701930710006316F70883274101F8
:1058300083A7870103278101B307F7002328F1001D
:10584000032701018327810163F0E70483274101D6
:105850000327010123A2E700832741010327410118
:1058600023A8E70097B70100938707DA03A707008B
:10587000832741019387470093850700130507009D
:10588000EFB08F846F000003130700009306000041
:10589000032681019305000003254101EFF05F8994
:1058A0002326A1008327C10063960700737004308C
:1058B0006F00000097B70100938707D583A7070003
:1058C00083A70700E39407F097B701009387C7D336
:1058D00083A70700232EF10097B70100938707D312
:1058E00003A7070097B70100938707D223A0E7001B
:1058F00097B70100938787D10327C10123A0E70051
:10590000130000008320C10213010103678000001F
:10591000130101FF23261100EFE01FD497B7010008
:10592000938707CF83A707006394070A17B5010081
:10593000130505CBEFA05FEA17B50100130585CB72
:10594000EFA09FE997B70100938707CC17B7010035
:10595000130707C923A0E70097B70100938707CB78
:1059600017B70100130707C923A0E70013060000BB
:105970009305000113054000EFB04F9E130705008B
:1059800097B701009387C7C823A0E70097B7010026
:10599000938707C883A707006396070073700430D6
:1059A0006F00000097B70100938787C683A70700A1
:1059B0006380070297B70100938787C583A7070015
:1059C00097A501009385056A13850700EFC04FBEB8
:1059D000EFE09FCC130000008320C1001301010100
:1059E00067800000130101FD232611022326A10078
:1059F0008327C100232EF1008327C100639607008F
:105A0000737004306F000000EFE01FC58327C101F1
:105A100083A74701B337F00093F7F70F232CF1006A
:105A2000EFE09FC783278101138507008320C10210
:105A30001301010367800000130101FD23261102F9
:105A40002326A1008327C100232EF1008327C10054
:105A500063960700737004306F000000EFE0DFBF53
:105A60008327C10183A70702232CF100EFE0DFC2E7
:105A700083278101138507008320C10213010103DD
:105A800067800000130101FD232611022326A100D7
:105A90002324B1008327C100232EF1008327C100F6
:105AA00063960700737004306F000000EFE0DFBA08
:105AB0008327C1010327810023A0E702EFE0DFBDB8
:105AC000130000008320C10213010103678000005E
:105AD000130101FC232E11022326A1002324B1006F
:105AE0002322C1002320D1009307E0FF232EF100E1
:105AF0008327C1002320F102832781002322F102A2
:105B0000832741002324F10297B70100938747B010
:105B100083A707001307C1019306000003260100B5
:105B20009305070013850700EFB0CFDF2326A102FE
:105B30008327C102138507008320C10313010104D9
:105B400067800000130101FC232E11022326A1000F
:105B50002324B1002322C1002320D10097B70100E4
:105B6000938707AB83A70700639607007370043021
:105B70006F0000009307F0FF232EF1008327C10080
:105B80002320F102832781002322F1028327410091
:105B90002324F10297B70100938787A783A7070003
:105BA0001307C101930600000326010093050700B7
:105BB00013850700EFB00FB32326A1028327C1028C
:105BC000138507008320C1031301010467800000CF
:105BD000130101FE232E11001305C001EF00D008B0
:105BE0002326A1008327C100638E07008327C100FD
:105BF00023A007008327C100938747001385070070
:105C0000EFA09FBD8327C100138507008320C1013A
:105C10001301010267800000130101FC232E110211
:105C20002326A1002324B1002322C1002320D10078
:105C30008327C1002324F10223220102032741000C
:105C4000B70700FFB377F70063860700737004306F
:105C50006F000000832741006396070073700430D3
:105C60006F000000EFE0CFF0930705006396070098
:105C70008327010063960700930710006F008000E0
:105C80009307000063960700737004306F000000F4
:105C9000EFD04F868327810283A707002320F102DC
:105CA000832581000325C100EF0080450327010201
:105CB000832781003367F70083274100B377F7001C
:105CC00003274100631CF702032701028327810099
:105CD000B367F7002326F1028327810203A7070099
:105CE0008327410093C7F7FF3377F70083278102AB
:105CF00023A0E700232001006F0040048327010058
:105D000063880702832781029386470003274100A7
:105D1000B7070005B367F700032601009385070066
:105D200013850600EFD05F90232601026F0000016B
:105D30008327810283A707002326F102EFC0DFFD3E
:105D4000232EA10083270100638407088327C10154
:105D500063940700EFA0DF83EFE0DF992326A10221
:105D60000327C102B7070002B377F700639807045F
:105D7000EFE09F8E8327810283A707002326F1028D
:105D80000327C10283274100B377F70003274100AF
:105D90006310F7028327810203A7070083274100CE
:105DA00093C7F7FF3377F7008327810223A0E7002B
:105DB000EFE09F8E930710002322F1020327C10218
:105DC000B70700019387F7FFB377F7002326F102A7
:105DD0008327C102138507008320C1031301010437
:105DE00067800000130101FB23261104232EA1006C
:105DF000232CB100232AC1002328D1002326E1004F
:105E00008327C101232AF102232C01022328010246
:105E10008327C10163960700737004306F00000090
:105E200003278101B70700FFB377F70063860700F8
:105E3000737004306F0000008327810163960700B0
:105E4000737004306F000000EFE08FD293070500FD
:105E5000639607008327C10063960700930710002D
:105E60006F00800093070000639607007370043092
:105E70006F000000EFC01FE88327410383A70700DE
:105E80002326F10203260101832581010325C10296
:105E9000EF00404F2324A10283278102638C070275
:105EA0008327C102232EF10223260100832741010B
:105EB000638807088327410303A70700832781011D
:105EC00093C7F7FF3377F7008327410323A0E70049
:105ED0006F0000078327C100639807008327C10272
:105EE000232EF1026F00C00583274101638A07005A
:105EF00003278103B7070001B367F700232CF102E2
:105F000083270101638A070003278103B707000481
:105F1000B367F700232CF1028327410393864700E0
:105F20000327810183278103B367F7000326C1009C
:105F30009385070013850600EFD00FEF232E010293
:105F4000EFC09FDD2322A1028327C10063880708D9
:105F50008327410263940700EFA08FE3EFE08FF9FE
:105F6000232EA1020327C103B7070002B377F7006E
:105F7000639C0704EFE04FEE8327410383A70700EC
:105F8000232EF10203260101832581010325C1038C
:105F9000EF00403F93070500638407028327410118
:105FA000638007028327410303A70700832781013A
:105FB00093C7F7FF3377F7008327410323A0E70058
:105FC000EFE08FED232801020327C103B70700018B
:105FD0009387F7FFB377F700232EF1028327C103DE
:105FE000138507008320C1041301010567800000A9
:105FF000130101FD232611022326A1002324B10051
:106000008327C100232EF1008327C1006396070078
:10601000737004306F00000003278100B70700FF92
:10602000B377F70063860700737004306F000000D9
:10603000EFE08FE28327C10183A70700232CF10043
:106040008327C10103A707008327810093C7F7FFB8
:106050003377F7008327C10123A0E700EFE0CFE308
:1060600083278101138507008320C10213010103E7
:1060700067800000130101FD232611022326A100E1
:106080002324B10093060000032681008325C1006C
:10609000170500001305852CEFF09FA3232EA10008
:1060A0008327C101138507008320C1021301010367
:1060B00067800000130101FD232611022326A100A1
:1060C0008327C100232EF100EFA0CFE39307050043
:1060D000232CF1008327C10183A70700232AF100A5
:1060E0008327810113850700EFA00FE0832741017B
:1060F000138507008320C10213010103678000009C
:10610000130101FB232611042326A1002324B1003F
:10611000232C01028327C1002328F102232A010234
:106120008327C10063960700737004306F0000007E
:1061300003278100B70700FFB377F70063860700E6
:10614000737004306F0000008327010393874700BA
:106150002326F1028327C102938787002324F102BB
:10616000EFC05FB98327C10283A7C700232EF102C6
:106170008327010303A70700832781003367F70004
:106180008327010323A0E7006F00000E8327C103CC
:1061900083A747002322F1028327C10383A70700B7
:1061A0002320F102232A010203270102B70700FF7F
:1061B000B377F700232EF10003270102B707000190
:1061C0009387F7FFB377F7002320F1020327C1017C
:1061D000B7070004B377F700639207028327010330
:1061E00003A7070083270102B377F700638807023C
:1061F00093071000232AF1026F0040028327010356
:1062000003A7070083270102B377F70003270102E2
:106210006316F70093071000232AF1028327410336
:10622000638007040327C101B7070001B377F700B4
:10623000638A07000327810383270102B367F700FE
:10624000232CF1028327010303A70700B7070002ED
:10625000B367F700938507000325C103EFD0CFE9AB
:1062600083274102232EF1020327C10383278102E2
:10627000E31EF7F08327010303A7070083278103A9
:1062800093C7F7FF3377F7008327010323A0E700C5
:10629000EFC09FA88327010383A70700138507008A
:1062A0008320C1041301010567800000130101FD73
:1062B000232611022326A1008327C100232EF100EB
:1062C0008327C10193874700232CF100EFC09FA2D1
:1062D0006F0040038327810103A7C7008327810143
:1062E000938787006316F700737004306F00000017
:1062F0008327810183A7C700B70500021385070024
:10630000EFD08FDF8327810183A70700E39407FC89
:106310000325C101EF000035EFC01FA013000000EE
:106320008320C1021301010367800000130101FEF5
:10633000232E11002326A1002324B10083258100F0
:106340000325C100EFF0DFDB130000008320C10153
:106350001301010267800000130101FE232E1100CA
:106360002326A1002324B100832581000325C10039
:10637000EFF01FC8130000008320C10113010102C8
:1063800067800000130101FE2326A1002324B10031
:106390002322C100232E01008327410063900702BE
:1063A0000327C10083278100B377F70063860702C4
:1063B00093071000232EF1006F0000020327C10095
:1063C00083278100B377F700032781006316F70066
:1063D00093071000232EF1008327C10113850700C6
:1063E0001301010267800000130101FD2326110241
:1063F0002326A1002324B1002322C10083264100CB
:10640000032681008325C10017050000130545F20E
:10641000EFF00FEC232EA1008327C10113850700A5
:106420008320C1021301010367800000130101FEF4
:106430002326A1008327C100232CF1008327C1005C
:1064400063960700232E01006F000001832781015E
:1064500083A78701232EF1008327C101138507003D
:106460001301010267800000130101FC232E1102B9
:106470002326A10023220102EFC0DF879737030004
:106480009387871A83A70700639C0700EF00002CFF
:1064900097370300938747191307100023A0E700DD
:1064A0008327C100638A07029307800013870700D0
:1064B0008327C100B387E7002326F1008327C100AB
:1064C00093F73700638A07008327C10093F7C7FF5C
:1064D000938747002326F1008327C10063820716B4
:1064E0000327C100B79701009387B7FF63EAE7145A
:1064F00097370300938747122324F102973703004D
:106500009387871183A707002326F1026F0080017C
:106510008327C1022324F1028327C10283A7070036
:106520002326F1028327C10283A747000327C10066
:1065300063F8E7008327C10283A70700E39A07FCFB
:106540000327C102973703009387870D630AF70E6D
:106550008327810283A7070013078000B387E70022
:106560002322F1028327C10203A7070083278102A8
:1065700023A0E7008327C10203A747008327C100A8
:10658000B307F74013078000131717006378F70865
:106590000327C1028327C100B307F700232EF100B0
:1065A0008327C10203A747008327C1003307F740B1
:1065B0008327C10123A2E7008327C1020327C1006B
:1065C00023A2E7008327C10183A74700232CF10002
:1065D00097370300938747042320F1026F000001DF
:1065E0008327010283A707002320F10283270102EA
:1065F00083A7070083A7470003278101E3E2E7FEA3
:106600008327010203A707008327C10123A0E70016
:10661000832701020327C10123A0E70097A70100F8
:10662000938747DD03A707008327C10283A747009D
:106630003307F74097A701009387C7DB23A0E70044
:10664000EFC08FED8327410263940700EF10801F96
:1066500083274102138507008320C103130101042E
:1066600067800000130101FD232611022326A100EB
:106670008327C100232CF1008327C1006382070A0E
:1066800093078000B307F04003278101B307F700A9
:10669000232CF10083278101232AF100EFC08FE52D
:1066A0008327410183A747002328F1009737030080
:1066B000938787F6232EF1006F0000018327C10125
:1066C00083A70700232EF1008327C10183A70700BA
:1066D00083A7470003270101E3E2E7FE8327C10107
:1066E00003A707008327410123A0E7008327C101F7
:1066F0000327410123A0E7008327410103A74700A7
:1067000097A70100938707CF83A707003307F700F8
:1067100097A70100938707CE23A0E700EFC0CFDF44
:10672000130000008320C1021301010367800000F1
:1067300097A70100938707CC83A70700138507005D
:10674000678000001300000067800000130101FF54
:1067500097A70100938787EC93F7C7FF2326F100E3
:1067600097370300938747EB0327C10023A0E70077
:1067700097370300938747EA23A207009737030060
:10678000938707EA379701001307C7FF23A2E700A3
:10679000973703009387C7E823A007008327C1002A
:1067A0002324F10083278100379701001307C7FFD7
:1067B00023A2E7008327810017370300130747E66A
:1067C00023A0E7001300000013010101678000000F
:1067D000130101FE2326A1002324B1002322C100BE
:1067E00083278100232EF1008327C100232CF10091
:1067F0000327C10083278100B367F70093F73700B1
:10680000639607066F00C0028327C10103A7070034
:106810008327810123A0E700832781019387470015
:10682000232CF1008327C10193874700232EF10019
:10683000832741009387D7FF0327C100B307F700E1
:1068400003278101E362F7FC6F0040020327C101C7
:1068500093071700232EF1008327810193861700E9
:10686000232CD100034707002380E7000327C10042
:1068700083274100B307F70003278101E368F7FC92
:106880008327C10013850700130101026780000000
:10689000130101FE2326A1002324B1002322C100FD
:1068A0000327C10083274100B367F70093F7370040
:1068B000639807068327810093F7F70F232AF100D7
:1068C000832741019397870003274101B367F700AE
:1068D000232AF100832741019397070103274101F0
:1068E000B367F700232AF1008327C100232EF100AC
:1068F0006F0080018327C10113874700232EE10029
:106900000327410123A0E7000327C100832741009B
:10691000B307F7000327C101E36EF7FC6F00C00364
:106920008327C100232CF1006F00C0018327810160
:1069300013871700232CE100032781001377F70F3B
:106940002380E7000327C10083274100B307F70036
:1069500003278101E36CF7FC8327C100138507003F
:106960001301010267800000130101FE2326A1002C
:106970008327C100232EF1006F0000018327C1018E
:1069800093871700232EF1008327C10183C70700D7
:10699000E39607FE0327C1018327C100B307F74031
:1069A000138507001301010267800000130101FE37
:1069B0002326A1002324B1008327C10013871700D9
:1069C0002326E10083C70700A30FF100832781007E
:1069D000138717002324E10083C70700230FF1006A
:1069E0008347F101638807000347F1018347E10111
:1069F000E304F7FC0347F1018347E101B307F740E4
:106A0000138507001301010267800000130101FED6
:106A10002326A1002324B1008327C100232EF100E7
:106A20001300000003278100930717002324F100BF
:106A30008327C10193861700232ED1000347070047
:106A40002380E70083C70700E39E07FC8327C1007C
:106A5000138507001301010267800000130101FE86
:106A60002326A100232E0100232C01006F0000012A
:106A70008327C100938717002326F1008327C100D5
:106A800003C7070093070002E304F7FE8327C10052
:106A900003C707009307D002630AF7008327C100EA
:106AA00003C707009307B0026312F7068327C100EC
:106AB00083C70700938737FD93B7170093F7F70F46
:106AC000232CF1008327C100938717002326F100B0
:106AD0006F00C0030327C1019307070093972700A6
:106AE000B387E70093971700232EF1008327C10097
:106AF000138717002326E10083C70700938707FD4C
:106B00000327C101B307F700232EF1008327C1003B
:106B100083C70700E39007FC832781016388070090
:106B20008327C101B307F0406F0080008327C101B4
:106B3000138507001301010267800000130101FEA5
:106B40002326A100973703009387C7AF83A70700C9
:106B500093861700173703001307C7AE2320D7000B
:106B60000327C1001377F70F97360300938686B18A
:106B7000B387F6002380E7000327C1009307A00036
:106B8000630CF700973703009387C7AB03A7070091
:106B900093070004631EF70497370300938787AEBB
:106BA000232EF1006F00C0038327C1011387170054
:106BB000232EE10003C70700B70710F0938707F003
:106BC00023A0E700973703009387C7A783A7070091
:106BD0001387F7FF973703009387C7A623A0E70023
:106BE00097370300938707A683A70700E39E07FA5A
:106BF000930700001385070013010102678000005E
:106C0000130101EB23261114232481142322911450
:106C100023202115232E3113232C4113232A511312
:106C2000232EA100232CB1002328C100232AD10048
:106C30002326E1002324F10023220101232601124F
:106C40008327C100138A0700930A000083270101EC
:106C50000328410113060A0093860A0013850700E2
:106C600093050800EF20C03F930705001388050037
:106C700013860700930608008327C11213871700A5
:106C80002326E112130706009397270093060113AA
:106C9000B387F60023AEE7EE8327C1001384070015
:106CA00093040000832741011387040063E8E7048D
:106CB00083274101138704006398E70083270101BC
:106CC0001307040063ECE7028327C1001389070060
:106CD00093090000130609009386090003250101AA
:106CE00083254101EF10105A930705001388050012
:106CF0002328F100232A01016FF09FF41300000004
:106D00006F0040018327C1018325810103254100D4
:106D1000E7800700832781001387F7FF2324E10022
:106D20000327C112E340F7FE6F0040058327C1121D
:106D30009397270013070113B307F70003A7C7EFC3
:106D40008327C1129397270093060113B387F60098
:106D500083A6C7EF9307900063F6D70093077005EB
:106D60006F00800093070003B387E7000327C1018A
:106D70008325810113850700E70007008327C112DF
:106D80001387F7FF2326E112E342F0FA1300000015
:106D90008320C11403248114832441140329011482
:106DA0008329C113032A8113832A41131301011577
:106DB00067800000130101FF2326A1002324B100F6
:106DC00083268100130710006356D7028327C10072
:106DD00083A707009387770093F787FF9386870041
:106DE0000327C1002320D70003A8470083A707007B
:106DF0006F00000503278100630407020327C10019
:106E000003270700130647008326C10023A0C600FE
:106E10000327070093070700130800006F004002D4
:106E20000327C10003270700130647008326C1007C
:106E300023A0C600032707009307070013080000DC
:106E40001385070093050800130101016780000006
:106E5000130101FF2326A1002324B1008326810012
:106E6000130710006356D7028327C10083A70700CA
:106E70009387770093F787FF938687000327C100E6
:106E80002320D70003A8470083A707006F008005D1
:106E900003278100630607020327C10003270700B9
:106EA000130647008326C10023A0C600032707005E
:106EB000930707001357F741130807006F0080027C
:106EC0000327C10003270700130647008326C100DC
:106ED00023A0C60003270700930707001357F741B5
:106EE000130807001385070093050800130101012B
:106EF00067800000130101FC232E1102232C810264
:106F0000232A91022326A1002324B1002322C100B9
:106F10002320D1006F0040026300043C832741001E
:106F2000938717002322F1008327C1008325810066
:106F300013050400E78007008327410083C707008B
:106F40001384070093075002E318F4FC83274100E1
:106F5000938717002322F100832741002328F100A3
:106F600093070002A30BF1009307F0FF232EF1001B
:106F70009307F0FF232CF100232001028327410017
:106F8000138717002322E10083C70700138407003B
:106F90009307D4FD130750056360F732139727005A
:106FA000979701009387070DB307F70003A7070022
:106FB000979701009387070CB307F70067800700D6
:106FC0009307D002A30BF1006FF05FFB9307000360
:106FD000A30BF1006FF09FFA232C0100032781011E
:106FE0009307070093972700B387E700939717004D
:106FF000B307F400938707FD232CF100832741009A
:1070000083C70700138407009307F00263D2870445
:107010009307900363CE870283274100938717006D
:107020002322F1006FF09FFB8327010013874700A5
:107030002320E10083A70700232CF1006F008001CB
:107040008327C101E3DC07F2232E01006FF01FF359
:10705000130000008327C101E3D207F283278101D7
:10706000232EF1009307F0FF232CF1006FF01FF1A6
:1070700083270102938717002320F1026FF01FF08E
:1070800083270100138747002320E10083A707001F
:107090000327C1008325810013850700E70007004F
:1070A0006F00402383270100138747002320E1005E
:1070B00083A407006396040097940100938404FB63
:1070C0008327C1016350F008034771019307D00281
:1070D000630AF7068327810193850700138504005F
:1070E000EF101018130705008327C101B387E7408D
:1070F000232EF1006F004002834771010327C10076
:107100008325810013850700E70007008327C1015D
:107110009387F7FF232EF1008327C101E34EF0FC94
:107120006F0040028327C1008325810013050400FE
:10713000E7800700938414008327C1019387F7FF3A
:10714000232EF10083C704001384070063000404A6
:1071500083278101E3C807FC832781019387F7FF19
:10716000232CF10083278101E3DE07FA6F00000280
:107170008327C1008325810013050002E7800700F3
:107180008327C1019387F7FF232EF1008327C101D5
:10719000E340F0FE6F000014930701008325010215
:1071A00013850700EFF0DFCA930705001388050079
:1071B0002324F10223260103832781020328C1022D
:1071C0009307080063D607048327C1008325810045
:1071D0001305D002E7800700832581020326C10240
:1071E0009307000013080000B386B740138506001C
:1071F00033B5A7003307C840B307A740138707007C
:1072000093870600130807002324F10223260103B5
:107210009307A0002322F1026F0040069307A0000D
:107220002322F1026F000004930780002322F10261
:107230006F004003930710002320F1028327C10051
:107240008325810013050003E78007008327C10021
:107250008325810013058007E7800700930700015D
:107260002322F10293070100832501021385070001
:10727000EFF05FB42324A1022326B10203274102C9
:1072800083477101138807008327C1010326810208
:107290008326C102832581000325C100EFF05F969C
:1072A0006F0040038327C10083258100130504007C
:1072B000E78007006F0000028327C100832581005B
:1072C00013055002E7800700832701012322F10004
:1072D000130000006FF05FC6130000008320C1039D
:1072E0000324810383244103130101046780000008
:1072F000130101FF2326A100B70710F0938707F2BF
:107300000327C10023A0E7006F000000130101FB69
:10731000232611022326A100232AB102232CC10215
:10732000232ED1022320E1042322F104232401058A
:107330002326110593070105938747FE232EF100AD
:107340008327C101938607000326C100930500002F
:1073500017F5FFFF1305C57EEFF0DFB993070000B7
:10736000138507008320C102130101056780000017
:10737000130101FE2326A1002324B1002322710062
:1073800083278100232EF1008327C10183A70700F3
:107390000327C1001377F70F2380E7008327C1017C
:1073A00083A70700138717008327C10123A0E700E5
:1073B000130000001301010267800000130101FAAD
:1073C000232E11022326A1002324B1002324C1046B
:1073D0002326D1042328E104232AF104232C0105C8
:1073E000232E1105930701062322F1029307410181
:1073F00093054101170600001306C6F737F7FFFF94
:107400009346F7FF37150000130505803388A50064
:107410003378E8001368783B23A007013305A60002
:107420003377E5001367773323A2E70033F7D500FE
:1074300093154701378703001307373933E7E50012
:1074400023A4E7003377D6009316470137070300DC
:107450001307770633E7E60023A6E7000F100000C6
:107460008327C1002326F10293070106938787FE35
:107470002324F102032781029307410113850700AA
:107480009307C10093060700032681009385070038
:10749000EFF05FA68327C100238007008327C10088
:1074A000138707008327C102B307F740138507003E
:1074B0008320C1031301010667800000130101FF4F
:1074C000370510F0130545F4032505002326A10018
:1074D000370510F0130505F4032505002324A1004A
:1074E000370510F0130545F4032505008328C10076
:1074F000E398A8FC0325C1001303050093030000D3
:10750000131703009306000003258100930505006F
:1075100013060000B3E7B6003368C700370710F062
:10752000130587F4B7150000938505FA13060000CC
:10753000B386B70093880600B3B8F8003307C800D5
:10754000B387E80013870700938706001308070036
:107550002320F5002322050113000000130101017F
:1075600067800000130101FF23261100EFF01FF5D3
:107570009307000873A04730130000008320C10068
:107580001301010167800000130101FE232E110089
:107590002326A10017950100130545C3EFF01FD75F
:1075A000130000008320C101130101026780000065
:1075B000130101FE232E11002326A10017950100BF
:1075C000130545C1EFF09FD4130000008320C101D3
:1075D0001301010267800000130101FD232611023F
:1075E0002326A100232E01006F004001130000009C
:1075F0008327C10193871700232EF1000327C101C0
:10760000B717000093877738E3D2E7FE179501009C
:107610001305C5BCEFF09FCF6FF0DFFC130101FD38
:10762000232611022326A100232E01006F00400112
:10763000EF10C01B8327C10193871700232EF10091
:107640000327C10193073001E3D4E7FE13000000D4
:107650008320C1021301010367800000130101FEB2
:10766000232E1100EF00402017070000130747FBEF
:1076700093060000130610009305200317950100E0
:10768000130545B6EFD09F9F2326A100EFB0DF85FD
:1076900093070500130700009306000013860700F8
:1076A000930510000325C100EFD09FA81300000030
:1076B0008320C1011301010267800000130101FE54
:1076C000232E110023260100EF10402D1307050083
:1076D00093071000630EF70017950100130505B11D
:1076E000EFF0DFC28327C10093E727002326F100D4
:1076F0008327C100138507008320C1011301010204
:1077000067800000130101FE232E110023260100D3
:10771000EFF0DFF417070000130787069306000059
:10772000130610009305400617950100130585AD5B
:10773000EFD0DF942326A1008327C10063820702D4
:10774000EFB08FFA930705001307000093060000BF
:1077500013860700930510000325C100EFD05F9D3D
:1077600023240100EFB04FCB9307000013850700DF
:107770008320C1011301010267800000130101FD94
:10778000232611022326A10097970100938787C51E
:1077900083A707001387470697970100938787C43D
:1077A00023A0E70097970100938707C483A70700EA
:1077B0001387470697970100938707C323A0E70025
:1077C00097970100938707C203A707009307F07CF0
:1077D00063DEE704979701009387C7C083A707007C
:1077E00013870783979701009387C7BF23A0E700FC
:1077F000EFF0DFEC232EA1008327C101639E070079
:1078000097970100938747BE03A70700B7170000AB
:107810009387F77663D0E7028327C10113850700BA
:10782000EFF01FADEFB04FCA6F0000011300000072
:107830006F008000130000008320C10213010103C8
:1078400067800000737004306F00000013000000B8
:1078500067800000130101FF2326A1002324B1004B
:10786000737004306F000000130101FE232E11001D
:107870009307C100930800001308000013071000CD
:1078800093060000130600409795010093854598E4
:10789000170500001305C530EFA08FEA8326C1004D
:1078A000930800001308000093070000130700006E
:1078B0001306004097950100938505961705000073
:1078C0001305050CEFA0CFE7930800001308000094
:1078D00097270300938747E01307100093064000A3
:1078E00013060040979501009385859317050000C6
:1078F0001305851DEFA0CFE49308000013080000D6
:1079000097270300938787DD1307100093068000F5
:107910001306004097950100938585901705000098
:107920001305851AEFA0CFE197270300938707DBA4
:1079300083A7070063960700737004306F00000090
:10794000EFE00FA91307050097270300938787D857
:1079500023A0E700972703009387C7D783A70700D3
:1079600063960700737004306F000000130000007E
:107970008320C1011301010267800000130101FD92
:10798000232611022326A1008327C100232CF10006
:10799000EFE00FA41307050097270300938747D351
:1079A00023A0E70097270300938787D283A70700C8
:1079B00063960700737004306F000000EF00104101
:1079C000232EA100EFE0CFA01307050097270300A7
:1079D000938707D023A0E70097270300938747CF1B
:1079E00083A7070063960700737004306F000000E0
:1079F000832581010325C101EF00500B232EA10037
:107A0000832581010325C101EF00C03F232EA10082
:107A1000972703009387C7CB83A707001385070029
:107A2000EFE0DF8803258101EFA09FA61307050083
:107A3000930730006306F70093071000232EF10030
:107A400097270300938747C983A70700138507007B
:107A5000EFA01FA413070500930730006306F7008B
:107A600093071000232EF10097270300938707C781
:107A700083A7070013850700EFA09FA11307050048
:107A8000930730006306F70093071000232EF100E0
:107A90008327C1016390070297270300938787C25A
:107AA00083A707001387170097270300938787C1D1
:107AB00023A0E7008327C101E38607F07370043039
:107AC0006F000000130101FD232611022326A100EF
:107AD000EF0090278327C100232EF100130500003B
:107AE000EFA01FD697270300938787BE83A70700C1
:107AF0009306F0FF1306F0008325C10113850700EC
:107B0000EFE08F91232CA1008327810113F7F70069
:107B10009307F0006306F700737004306F000000F5
:107B200013050000EFA0DFD197270300938747BA22
:107B300083A707009306F0FF1306F0008325C10119
:107B400013850700EFE04F8D232CA10083278101CF
:107B500013F7F7009307F0006306F7007370043023
:107B60006F00000097270300938787B683A707005D
:107B70001307F0FF93061000130600009305F000B2
:107B800013850700EFE00FA6232CA10083278101B6
:107B9000E38607F4737004306F000000130101FDE9
:107BA000232611022326A100232E01001305000025
:107BB000EFA01FC997270300938787B183A707000A
:107BC0001307F0FF93061000130610009305200022
:107BD00013850700EFE00FA1232CA10003278101EB
:107BE0009307200A6306F70093071000232EF10085
:107BF000972703009387C7AD83A707001307F0FFFC
:107C000093061000130600009305200A1385070051
:107C1000EFE04F9D232CA1008327810113F7270A52
:107C20009307200A6306F70093071000232EF10044
:107C300013050000EFA0DFC097270300938747A933
:107C400083A707001307F0FF930610001306100028
:107C50009305200A13850700EFE0CF98232CA1009D
:107C6000032781019307F00F6306F70093071000C5
:107C7000232EF10013050000EFA09FBC97270300FF
:107C8000938707A583A707009306F0FF1306F0006C
:107C90009305200013850700EFD01FF8232CA100C7
:107CA0008327810113F7F7009307F0006306F700BD
:107CB00093071000232EF10097270300938747A115
:107CC00083A707009305000013850700EFE04FC36B
:107CD000930705006386070093071000232EF10029
:107CE000972703009387C79E83A70700930500008B
:107CF00013850700EFE0CFAF930705006386070009
:107D000093071000232EF1008327C101639007021F
:107D1000972703009387479B83A7070013871700C4
:107D2000972703009387479A23A0E70013050000D5
:107D3000EFA01FB1972703009387879983A70700B8
:107D40009306F0FF1306F00093052000138507004B
:107D5000EFD09FEC232CA1008327810113F7F700BC
:107D60009307F0006306F70093071000232EF1003D
:107D7000972703009387C79583A707009305000003
:107D800013850700EFE0CFB7930705006386070070
:107D900093071000232EF100972703009387479342
:107DA00083A707001307F0FF9306100013060000D7
:107DB0009305F00013850700EFE0CF82232CA1008C
:107DC000832781016386070093071000232EF100AB
:107DD0008327C10163900702972703009387C78E0B
:107DE00083A7070013871700972703009387C78D82
:107DF00023A0E7008327C101E38A07DA7370043008
:107E00006F000000130101FD232611022326A100AB
:107E10002324B10003258100EFA08FE7130705009D
:107E2000930730006306F700930710002326F10044
:107E3000972703009387478A83A7070013850700C6
:107E4000EFA00FE513070500930730006306F70066
:107E5000930710002326F1009727030093870788D4
:107E600083A7070013850700EFA08FE21307050023
:107E7000930730006306F700930710002326F100F4
:107E8000972703009387C78483A707009305E00023
:107E900013850700EFE0CFA697270300938747835A
:107EA00083A707009306F0FF130610009305100048
:107EB00013850700EFD05FD6232EA1008327C101D1
:107EC00093F7170063960700930710002326F1002D
:107ED000971703009387C77F83A7070093050000C8
:107EE00013850700EFE0CF90130705009307E0002C
:107EF0006306F700930710002326F100971703008D
:107F00009387077D83A707009305E000138507008B
:107F1000EFE00F8E971703009387877B83A70700F7
:107F20009305000013850700EFE08F8C9307050091
:107F300063860700930710002326F10003258100C4
:107F4000EFA0DFAA971703009387077983A707009D
:107F500013850700EFA09FA9971703009387077861
:107F600083A7070013850700EFA05FA80325810002
:107F7000EFA00FD213070500930720006306F70058
:107F8000930710002326F100971703009387C77407
:107F900083A7070013850700EFA08FCF1307050005
:107FA000930720006306F700930710002326F100D3
:107FB000971703009387877283A70700138507002D
:107FC000EFA00FCD13070500930720006306F7000D
:107FD000930710002326F100971703009387476F3C
:107FE00083A707009306F0FF1306F0009305100027
:107FF00013850700EFD05FC2232EA1008327C101A4
:1080000013F7F7009307F0006306F70093071000DB
:108010002326F100971703009387876B83A7070038
:108020009305000013850700EFD09FFC9307050020
:1080300063860700930710002326F10003258100C3
:10804000EFA00FC513070500930730006306F70084
:10805000930710002326F100971703009387C76743
:1080600083A7070013850700EFA08FC21307050041
:10807000930730006306F700930710002326F100F2
:10808000971703009387876583A707001385070069
:10809000EFA00FC013070500930730006306F70039
:1080A000930710002326F10003258100EFA01F9401
:1080B000971703009387476283A70700138507007C
:1080C000EFA0DF92971703009387476183A707000C
:1080D00013850700EFA09F9103258100EFA04FBB00
:1080E00013070500930720006306F70093071000AD
:1080F0002326F100971703009387075E83A70700E5
:1081000013850700EFA0CFB81307050093072000E1
:108110006306F700930710002326F100971703006A
:108120009387C75B83A7070013850700EFA04FB6AF
:1081300013070500930720006306F700930710005C
:108140002326F1009305200013050000EFA00FCFB8
:10815000971703009387C75783A707009306F0FF7D
:108160001306F0009305100013850700EFD0DFAA77
:10817000232EA1008327C10113F7F7009307F00016
:108180006306F700930710002326F10097170300FA
:108190009387075483A70700930500001385070002
:1081A000EFD01FE5930705006386070093071000D3
:1081B0002326F10003258100EFA08FAD13070500F2
:1081C000930710006306F700930710002326F100C1
:1081D000971703009387475083A70700138507006D
:1081E000EFA00FAB13070500930710006306F7001D
:1081F000930710002326F100971703009387074E7B
:1082000083A7070013850700EFA08FA813070500B9
:10821000930710006306F700930710002326F10070
:108220009305000013050000EFA04FC10325810056
:10823000EFA00FA613070500930720006306F700C1
:10824000930710002326F100971703009387C74870
:1082500083A7070013850700EFA08FA3130705006E
:10826000930720006306F700930710002326F10010
:10827000971703009387874683A707001385070096
:10828000EFA00FA113070500930720006306F70076
:10829000930710002326F1008327C10013850700F0
:1082A0008320C1021301010367800000130101FD57
:1082B000232611022326A1002324B10003258100D7
:1082C000EFA0CFF203258100EFA08F9C13070500DC
:1082D000930720006306F700930710002326F100A0
:1082E000971703009387C73E83A707009305200ACB
:1082F00013850700EFD0DFE0971703009387473D12
:1083000083A7070013070000930600001306000070
:108310009305F00F13850700EFD0DFAC232EA100EB
:108320000327C1019307000A6306F70093071000B3
:108330002326F10003258100EFA08F951307050088
:10834000930720006306F700930710002326F1002F
:10835000971703009387C73783A707009305D00FAC
:1083600013850700EFD0DFD99717030093874736AF
:1083700083A7070013070000930600001306000000
:108380009305F00F13850700EFD0DFA5232EA10082
:108390000327C1019307D00F6306F700930710006E
:1083A0002326F10003258100EFA08F8E130705001F
:1083B000930720006306F700930710002326F100BF
:1083C000971703009387C73083A707009305200002
:1083D00013850700EFD0DFD203258100EFA04F8B7C
:1083E00013070500930730006306F700930710009A
:1083F0002326F100971703009387872D83A7070093
:108400009305000013850700EFD09FCF13070500E9
:108410009307F00F6306F700930710002326F1007F
:10842000971703009387C72A83A7070093052000A7
:1084300013850700EFD0DFBB130705009307F00F8C
:108440006306F700930710002326F100032581003F
:10845000EFA0CFD903258100EFA08F83130705007C
:10846000930720006306F700930710002326F1000E
:10847000971703009387C72583A70700930520005C
:1084800013850700EFD0DFC703258100EFA04F80E1
:1084900013070500930730006306F70093071000E9
:1084A0002326F100971703009387872283A70700ED
:1084B0001307000093060000130600009305F00F59
:1084C00013850700EFD01F92232EA1000327C101BF
:1084D0009307D0056306F700930710002326F100E9
:1084E000971703009387C71E83A707009305F00F14
:1084F00013850700EFD0DFAF130705009307D00502
:108500006306F700930710002326F1009717030076
:108510009387071C83A707009305000013850700B6
:10852000EFD01FAD93070500638607009307100087
:108530002326F1008327C100138507008320C10291
:108540001301010367800000130101FE232E1100B7
:10855000EFB0DFDF13070500971703009387C717F6
:1085600083A707006318F700930730002326F10064
:108570006F00C000930750002326F1001305000090
:10858000EFA00FAC971703009387871483A707000A
:108590001307F0FF93060000130610008325C100A7
:1085A00013850700EFD01F842324A10083278100B7
:1085B000638407006FF09FFC1300000013000000AD
:1085C0008320C1011301010267800000130101FE35
:1085D000232E110023260100971703009387C70F4E
:1085E00083A7070013850700EF909FEA1307050094
:1085F000930730006306F700930710002326F1006D
:10860000971703009387870D83A70700138507003B
:10861000EF901FE813070500930730006306F7008B
:10862000930710002326F100930710002324F10084
:108630006F000016971703009387070A83A70700A8
:1086400013850700EFA08FBA9717030093870709D8
:1086500083A7070013850700EFA04FB99717030002
:108660009387870783A7070013850700EF905FE2D2
:1086700013070500930720006306F7009307100017
:108680002326F100971703009387470583A7070068
:1086900013850700EF90DFDF130705009307200025
:1086A0006306F700930710002326F10097170300D5
:1086B0009387070283A7070083258100138507009E
:1086C000EFD01FA48327810093F737006398070238
:1086D000971703009387470083A7070013850700B8
:1086E000EF901FDB1307050093072000630CF702D0
:1086F000930710002326F1006F00C00297170300B4
:10870000938787FD83A7070013850700EF905FD845
:1087100013070500930730006306F7009307100066
:108720002326F1008327810093F7570063980702FF
:1087300097170300938787FA83A70700138507001D
:10874000EF901FD51307050093072000630CF70275
:10875000930710002326F1006F00C0029717030053
:108760009387C7F783A7070013850700EF905FD2B1
:1087700013070500930730006306F7009307100006
:108780002326F10083278100939717002324F1000B
:10879000032781009307F00FE3FEE7E89717030034
:1087A000938787F383A7070013850700EFA00FA423
:1087B00097170300938787F283A7070013850700A5
:1087C000EFA0CFA297170300938787F083A7070036
:1087D00013850700EFD09FAD8327C10013850700E5
:1087E0008320C1011301010267800000130101FD14
:1087F0002326110293074006232EF1009307800CD5
:10880000232CF1009307C012232AF10093072001C3
:108810002328F10097170300938787EC83A70700AD
:108820001387170097170300938787EB23A0E700B0
:10883000971703009387C7EA83A707000327C1019F
:10884000631CF706971703009387C7E883A7070001
:1088500013850700EFD01F862326A1008327C100C0
:10886000638C0700971703009387C7E7130710006F
:1088700023A0E7006F00801197170300938787E517
:1088800083A7070013060000832501011385070055
:10889000EFD09FB52324A100032781009307100088
:1088A0006306F70E971703009387C7E313071000BB
:1088B00023A0E7006F00800D97170300938747E21E
:1088C00083A7070003278101631EF70297170300A0
:1088D000938747E083A7070013850700EFD08FFD3C
:1088E0002326A1000327C100832701016300F70AA3
:1088F00097170300938707DF1307100023A0E700F3
:108900006F00C00897170300938787DD83A70700D0
:1089100003274101631CF70697170300938787DB42
:1089200083A707008325010113850700EFD08FF48B
:10893000930705002326F1000327C10093071000C9
:10894000630AF700971703009387C7D9130710002E
:1089500023A0E70097170300938787D823A0070079
:1089600097170300938707D883A707006390070230
:1089700097170300938787D583A7070013871700EE
:1089800097170300938787D423A0E7001300000004
:108990008320C1021301010367800000130101FF5E
:1089A000930710002326F100971703009387C7D37E
:1089B00003A70700971703009387C7D083A7070073
:1089C0006314F7002326010097170300938787CFCE
:1089D00003A7070097170300938707D123A0E70099
:1089E00097170300938787D003A707009717030003
:1089F000938787CD83A707006314F7002326010020
:108A000097170300938747CC03A707009717030026
:108A10009387C7CD23A0E70097170300938747CD1F
:108A200003A7070097170300938747CA83A7070088
:108A30006314F7002326010097170300938707C9E3
:108A400003A7070097170300938787CA23A0E700AF
:108A50008327C1001385070013010101678000000F
:108A6000B305B500930705006386B70003C7070089
:108A7000631607003385A7406780000093871700BF
:108A80006FF09FFE130101FD23229102232A510161
:108A9000232611022324810223202103232E3101C6
:108AA000232C410123286101232671012324810104
:108AB000232291012320A101930A0500938405003C
:108AC000639E063813040600930905001779010018
:108AD0001309897563F8C512B7070100138B0500E8
:108AE0006378F6101307F00F3337C70013173700FA
:108AF000B357E6003309F900834609003387E600DF
:108B000093060002B386E640638C0600B394D4005B
:108B100033D7EA003314D600336B9700B399DA00E9
:108B2000935A040193850A0013050B00EF00902A65
:108B30001309050093850A00931B040113050B001C
:108B4000EF00D02493DB0B0193040500930505008F
:108B500013850B00EF00D0201319090193D70901E9
:108B6000B367F900138A040063FEA700B387870088
:108B7000138AF4FF63E8870063F6A700138AE4FF13
:108B8000B3878700B384A74093850A001385040048
:108B9000EF0050241309050093850A001385040093
:108BA000EF00D01E93990901930405009305050079
:108BB0001319090113850B0093D90901EF00501A0D
:108BC000B36939011386040063FCA900B3093401B9
:108BD0001386F4FF63E6890063F4A9001386E4FFBB
:108BE00013140A013364C400130A00006F00001359
:108BF000B707000113070001E36CF6EE13078001CD
:108C00006FF01FEF138A0600631A06009305000039
:108C100013051000EF00901713040500B7070100BB
:108C2000637EF4129307F00F63F48700130A800049
:108C3000B35744013309F9000347090093060002C2
:108C400033074701B386E64063940612B384844039
:108C5000130A1000135B040193050B001385040035
:108C6000EF0050171309050093050B00138504004E
:108C7000931B0401EF00901193DB0B01930405009B
:108C80009305050013850B00EF00900D13190901E2
:108C900093D70901B367F900938A040063FEA70024
:108CA000B3878700938AF4FF63E8870063F6A70021
:108CB000938AE4FFB3878700B384A74093050B0032
:108CC00013850400EF0010111309050093050B0034
:108CD00013850400EF00900B93990901930405009C
:108CE000930505001319090113850B0093D9090198
:108CF000EF001007B36939011386040063FCA90073
:108D0000B30934011386F4FF63E6890063F4A90014
:108D10001386E4FF13940A013364C40013050400AE
:108D200093050A008320C1020324810283244102A7
:108D3000032901028329C101032A8101832A4101F8
:108D4000032B0101832BC100032C8100832C4100E4
:108D5000032D01001301010367800000B707000124
:108D6000130A0001E366F4EC130A80016FF05FEC74
:108D70003314D40033DAE400B399DA0033D7EA00CD
:108D8000935A0401B394D40093850A0013050A0092
:108D9000336B9700EF0010041309050093850A0058
:108DA00013050A00931B0401EF00407E93DB0B01C7
:108DB000930405009305050013850B00EF00407A2E
:108DC0001319090113570B013367E900138A0400D3
:108DD000637EA70033078700138AF4FF6368870068
:108DE0006376A700138AE4FF33078700B304A74024
:108DF00093850A0013850400EF00C07D1309050068
:108E000093850A0013850400EF0040789304050061
:108E10009305050013850B00EF00807413170B01F9
:108E20001357070113190901B367E90013870400F9
:108E300063FEA700B38787001387F4FF63E887000A
:108E400063F6A7001387E4FFB3878700131A0A01AC
:108E5000B384A740336AEA006FF0DFDF63ECD51E0E
:108E6000B707010063F4F6041307F00FB335D7001A
:108E70009395350033D7B600977701009387C73AAB
:108E8000B387E70003C70700130A00023307B700E0
:108E9000330AEA4063160A0213041000E3E096E87E
:108EA00033B6CA00134416006FF05FE7B70700013E
:108EB00093050001E3E0F6FC930580016FF09FFB52
:108EC000B35CE600B3964601B3ECDC0033D4E400B7
:108ED00093DB0C01B397440133D7EA0093850B0071
:108EE00013050400336BF700B3194601EF00806EE1
:108EF0001309050093850B0013050400139C0C0156
:108F0000EF00C068135C0C01930405009305050095
:108F100013050C00EF00C0641319090113570B016E
:108F20003367E90013840400637EA70033079701C9
:108F30001384F4FF636897016376A7001384E4FF4A
:108F400033079701B304A74093850B0013850400F2
:108F5000EF0040681309050093850B00138504009A
:108F6000EF00C062930405009305050013050C0093
:108F7000EF00005F93170B011319090193D7070145
:108F8000B367F9001386040063FEA700B387970157
:108F90001386F4FF63E8970163F6A7001386E4FFE6
:108FA000B387970113140401B70B01003364C400A5
:108FB0001389FBFF337D240133F92901B384A740D2
:108FC0009305090013050D00EF008059935C04011F
:108FD00093050900130B050013850C00EF004058A2
:108FE00093D90901130C05009385090013850C0022
:108FF000EF000057130905009385090013050D00C4
:10900000EF0000563305850193570B013385A70008
:10901000637485013309790193570501B3872701EB
:1090200063E6F402E392F4BCB70701009387F7FF0D
:109030003375F50013150501337BFB0033964A01A8
:1090400033056501130A0000E37AA6CC1304F4FF8C
:109050006FF09FB9130A0000130400006FF01FCCDB
:10906000130101FB2324810423229104232E3103C5
:10907000232291032326110423202105232C4103BD
:10908000232A510323286103232671032324810308
:109090002320A103232EB101930C05009389050021
:1090A0001304050093840500639E06261309060039
:1090B000138A0600977A0100938A0A1763F4C5148D
:1090C000B70701006376F6129307F00F63F4C70049
:1090D000130A8000B3574601B38AFA0003C70A0097
:1090E0001305000233074701330AE540630C0A0009
:1090F000B395490133D7EC0033194601B364B70087
:1091000033944C01935A090193850A001385040096
:10911000EF00404C9309050093850A00131B0901D9
:1091200013850400EF008046135B0B0193050500D7
:1091300013050B00EF00C0429399090193570401F6
:10914000B3E7F90063FAA700B387270163E62701B5
:1091500063F4A700B3872701B384A74093850A006F
:1091600013850400EF0000479309050093850A006A
:1091700013850400EF0080411314040193050500DA
:109180009399090113050B0013540401EF00403DAE
:1091900033E48900637AA400330424016366240164
:1091A0006374A400330424013304A4403355440100
:1091B000930500008320C104032481048324410417
:1091C000032901048329C103032A8103832A41035C
:1091D000032B0103832BC102032C8102832C410248
:1091E000032D0102832DC1011301010567800000D9
:1091F000B7070001130A0001E36EF6EC130A8001C1
:109200006FF05FED631A0600930500001305100070
:10921000EF00C03713090500B7070100637AF90EA4
:109220009307F00F63F42701130A8000B357490135
:10923000B38AFA0003C70A0013050002B384294168
:1092400033074701330AE540E30E0AEA33194901BF
:10925000B3DAE900B395490133D7EC00935409011F
:10926000336BB70013850A0093850400EF00803646
:109270009309050093850400931B090113850A00D7
:10928000EF00C03093DB0B019305050013850B0045
:10929000EF00002D9399090193570B01B3E7F900F3
:1092A00033944C0163FAA700B387270163E62701D3
:1092B00063F4A700B3872701B38AA740938504000E
:1092C00013850A00EF00003193090500938504001F
:1092D00013850A00EF00802B9305050013850B0012
:1092E000EF00002893150B019399090193D505010F
:1092F000B3E5B90063FAA500B385250163E625014E
:1093000063F4A500B3852501B384A5406FF09FDF0A
:10931000B7070001130A0001E36AF9F0130A80019C
:109320006FF0DFF0E3E8D5E8B707010063FCF6046F
:10933000930BF00F33B5DB001315350033D7A600C0
:1093400097770100938747EEB387E70083CB070049
:1093500093050002B38BAB00338B7541631E0B0288
:1093600063E4360163EACC003384CC40B386D94051
:1093700033B58C00B384A640130504009385040024
:109380006FF05FE3B707000113050001E3E8F6FAA9
:10939000130580016FF09FFAB3966601335D760185
:1093A000336DDD0033D47901B395690133DC7C0181
:1093B00093540D01336CBC00130504009385040025
:1093C000B31A6601EF000021130A0500938504001B
:1093D0001305040033996C01931C0D01EF00001B71
:1093E00093DC0C01130405009305050013850C00A4
:1093F000EF000017131A0A0113570C013367EA0034
:10940000130A0400637EA7003307A701130AF4FFC1
:109410006368A7016376A700130AE4FF3307A70177
:10942000B309A7409385040013850900EF00801A53
:10943000938504001304050013850900EF0000154F
:10944000930505009304050013850C00EF004011FF
:1094500093150C011314040193D50501B365B400F1
:109460001387040063FEA500B385A5011387F4FFED
:1094700063E8A50163F6A5001387E4FFB385A501A2
:10948000131A0A01B70C0100336AEA001384FCFFC7
:10949000B3778A0033F48A00B384A54013850700AC
:1094A000930504002326F100135A0A01EF00400B34
:1094B000930905009305040013050A00EF00400A14
:1094C00013DC0A01930D050093050C0013050A0037
:1094D000EF0000098327C100130A050093050C0063
:1094E00013850700EF00C0073305B50113D7090145
:1094F0003307A7006374B701330A9A01B707010065
:109500009387F7FF935507013377F7001317070188
:10951000B3F7F900B3854501B307F70063E6B4007C
:10952000639EB400637CF90033865741B3B7C7002C
:10953000B385A541B385F54093070600B307F9400D
:109540003339F900B385B440B385254133947501AF
:10955000B3D767013365F400B3D565016FF09FC5DC
:10956000130605001305000093F61500638406003A
:109570003305C50093D5150013161600E39605FEB6
:10958000678000006340050663C605061386050074
:10959000930505001305F0FF630C06029306100007
:1095A000637AB6006358C00013161600939616002F
:1095B000E36AB6FE1305000063E6C500B385C54047
:1095C0003365D50093D6160013561600E39606FEB3
:1095D0006780000093820000EFF05FFB13850500B9
:1095E000678002003305A04063D80500B305B04092
:1095F0006FF0DFF9B305B04093820000EFF01FF980
:109600003305A040678002009382000063CA050012
:10961000634C0500EFF09FF713850500678002009B
:10962000B305B040E35805FE3305A040EFF01FF648
:089630003305B0406780020021
:02000004800278
:1000000049444C4500000000244BFEFFBC4AFEFF63
:10001000D84AFEFFF04AFEFF004BFEFFF44CFEFF05
:100020008C4CFEFFA84CFEFFC04CFEFFD04CFEFFE8
:10003000546D7220537663006456FEFF6456FEFFD3
:100040006456FEFF4C57FEFFF456FEFF3C57FEFF82
:100050006456FEFF6456FEFF4C57FEFFF456FEFF4B
:10006000546D725100000000286E756C6C29000000
:100070000C6FFEFF4872FEFF3472FEFF4872FEFFF7
:100080004872FEFF4872FEFF4872FEFFB86FFEFF27
:100090004872FEFF4872FEFF506FFEFFD06FFEFFFA
:1000A0004872FEFF5C6FFEFF686FFEFF686FFEFF29
:1000B000686FFEFF686FFEFF686FFEFF686FFEFFF0
:1000C000686FFEFF686FFEFF686FFEFF4872FEFFFD
:1000D0004872FEFF4872FEFF4872FEFF4872FEFF44
:1000E0004872FEFF4872FEFF4872FEFF4872FEFF34
:1000F0004872FEFF4872FEFF4872FEFF4872FEFF24
:100100004872FEFF4872FEFF4872FEFF4872FEFF13
:100110004872FEFF4872FEFF4872FEFF4872FEFF03
:100120004872FEFF4872FEFF4872FEFF4872FEFFF3
:100130004872FEFF4872FEFF4872FEFF4872FEFFE3
:100140004872FEFF4872FEFF4872FEFF4872FEFFD3
:100150004872FEFF4872FEFF4872FEFF4872FEFFC3
:100160004872FEFF4872FEFF4872FEFF4872FEFFB3
:100170001070FEFF2871FEFF4872FEFF4872FEFFFE
:100180004872FEFF4872FEFF4872FEFF4872FEFF93
:100190004872FEFF0070FEFF4872FEFF4872FEFFCD
:1001A000B871FEFFC471FEFF4872FEFF4872FEFF89
:1001B0003470FEFF4872FEFFAC71FEFF4872FEFF16
:1001C0004872FEFFEC71FEFF6D69616F750A0000F9
:1001D0006D69616F75320A0068756E6772790A0021
:1001E00054696D65723200004572726F7220696EDB
:1001F00020787878207461736B73200D0A000000FA
:10020000436865636B54696D65720000576169747A
:100210004F0000005365744200000000526E647687
:1002200000000000000102020303030304040404AD
:100230000404040405050505050505050505050572
:100240000505050506060606060606060606060652
:10025000060606060606060606060606060606063E
:100260000606060607070707070707070707070722
:10027000070707070707070707070707070707070E
:1002800007070707070707070707070707070707FE
:1002900007070707070707070707070707070707EE
:1002A00007070707080808080808080808080808D2
:1002B00008080808080808080808080808080808BE
:1002C00008080808080808080808080808080808AE
:1002D000080808080808080808080808080808089E
:1002E000080808080808080808080808080808088E
:1002F000080808080808080808080808080808087E
:10030000080808080808080808080808080808086D
:10031000080808080808080808080808080808085D
:0403200008080808B9
:100324001000000000000000017A5200017C01016D
:100334001B0D02004C000000180000004487FEFF63
:10034400DC05000000440E307089039507810188A4
:100354000292049305940696089709980A990B9AB1
:100364000C0370020AC144C844C944D244D344D4DF
:1003740044D544D644D744D844D944DA440E00443E
:100384000B0000005000000068000000D08CFEFF4D
:100394000005000000440E507488028903930599F7
:1003A4000B810192049406950796089709980A9A76
:1003B4000C9B0D0320010AC144C844C944D244D350
:1003C40044D444D544D644D744D844D944DA44DB4D
:0803D400440E00440B00000080
:1003E800AAAAAAAA08000000FC8F010009000000C0
:040000058000004037
:00000001FF
